:020000040000fa
:080000001401040000000000df
:020000040000fa
:10020000140104000000000094010400000000003c
:10021000c2010400000000000e0b040000000000fa
:100220000000040000000000cfd7200080792200e9
:100230000001880000000000050007000c00070016
:100240006a280200000000000040da000000fe0002
:100250004440a900c02121000000e000030032005a
:1002600000002000a00188004440a8000000060013
:100270002005250001002000160037006200400024
:10028000e0804800910188009001ba0062004000bf
:10029000e0804800910188009002ba0062004000ae
:1002a000e08048000002eb006028e10005003a0011
:1002b0008301e90007003300038009000059eb00c7
:1002c000040037006128e100010032000082eb00e9
:1002d00005000700910188001001ba000200e0004b
:1002e000e6ff3a00000005009101880080027800d6
:1002f00062004000e08048003559ba008301e900ff
:10030000080032002559ba008301e90005003200d7
:100310000400e000f4ff320015d9ba008301e900bf
:10032000f1ff3a0000000600881f78000204780000
:1003300082000700080040004f047800000006001b
:100340000000fa00881f7800000478003fb9970089
:10035000ea81570080007800401920007e000700e5
:10036000800078000000e000020035000040eb0053
:1003700000f47800010078004f0478000080fa0053
:1003800000000600889fbe0080047800010078000d
:100390000204780089017800110020000f00070096
:1003a00089007800880f5000010032008000eb00c7
:1003b000010078004f04be00000006000000fa00b3
:1003c0004fb99700e8815700219e2000201c200093
:1003d000610007000080fa0000000600e487470083
:1003e000889fbe008a9fbe008c9fbe008e1f780033
:1003f00081bf9f00820078008304780000077800a6
:100400000fb997000116b8008c0578000001eb00c9
:100410000c00e00042003200010178008fb9970023
:100420000300e0003e0032000c00e0002e0032002d
:10043000c900900069009000808f500004003900ce
:1004400009007800f90007000000e00026003500f0
:1004500019a8a300060032000b017800a1002000bb
:100460000e00780036010700000578000100370013
:100470000005eb000b0478000a00e00002003200e7
:100480000e0055000004e80069009000c9019000ca
:1004900003005000880f5000020031000005eb00ff
:1004a00000047800080178008e00780003007800ce
:1004b0002200070008074700888555004900900082
:1004c00008004000c00498000a00e0000400320068
:1004d00009007800230107000000e00002003a0054
:1004e0000b00e000d2ff3a0019b8a300020032006e
:1004f000090078001b01070000c0200019006000ff
:100500000200320049009000e00498000b00560001
:100510008fb99700110009000380d800000178000e
:10052000020078004f0778004f06be004f05be005e
:100530004f04be004f00b1000000060080017800ab
:100540000200e00003003200b15978000201e90026
:10055000fdff3a00000006006200fa00889fbe001e
:100560008a9fbe000004be00020578008300780068
:100570006a80570037010700f88f9f0089979f0016
:100580000000eb00909f9f001a80fb008005fb009d
:100590000000ea00cf04de000904780050022000c9
:1005a000808f550001003a000904e9000800e000ce
:1005b0000c0034000f909700080178008a00780042
:1005c000ff8997000300010080979f008080eb0067
:1005d0000000e000900032001f98970008004000e3
:1005e000909f9f000905450050022000808f550014
:1005f000040032000b00e000e3ff3a009f989700f0
:10060000850037000000eb00f0979f00e0979f0007
:10061000d0979f00c0979f00b0979f00a0979f0022
:10062000b09f9f000900370040b1200000805000bb
:100630000000d000a1b1200001004000bf98970049
:1006400090807000b19f9f000a05e8009a00fb00af
:1006500040b1200001010700800078000000e000a8
:10066000f1ff3a00a0c2b3009a4f10000e003a000a
:100670003fb897000080e900b0bf9f0010007800ed
:10068000a09f9f000000e00005003d000000ea0080
:10069000a09f9f003f9897000020a000b09f9f0060
:1006a0000a05e80011003700a19f9f000b003700ea
:1006b000af989700f0ff2700808f500006003200af
:1006c0006a09b9001a00fb000200400001fd2f007a
:1006d00001004000a09f9f000a05e8001a00fb00ef
:1006e000e60007000000e000f1ff3a00e0c2b300be
:1006f0009a4f1000030032000080eb00809f9f00a3
:100700001c003700a0c2b300da4f100007003a0007
:100710003fb897000080e900b0bf9f00100078004c
:10072000809f9f000a05e800120037000000eb00e0
:10073000809f9f000b0037008f989700f0ff2700e5
:10074000808f5000060032006a09b9001a00fb00d1
:100750000200400001fd2f0001004000809f9f002b
:100760000a05e8001a00fb00c40007000000e000d2
:10077000f1ff3a009a00fb00e0b72000b700070045
:100780008040eb000000e00001003200ba40780039
:10079000817f9f0080c6b30080cf500004003a00e4
:1007a0009acf100002003a00664050000700370060
:1007b0008f789700c0c6b30080cf500005003a0084
:1007c0009acf100003003a0065404000807f9f00f0
:1007d0000a05e800a0fb2f00008447003a4178009a
:1007e00088017800ea80570060f92f000f00400070
:1007f000760107000000e00006003a00880078005b
:1008000060f92f000f004000a20007000000e00088
:100810005dff3d008080eb00010078004f05be00c9
:100820004f04be000080fa0000000600889fbe0052
:1008300000047800c0019000600090008000eb0090
:10084000808f51003b0039001801780020002900fa
:1008500000006100e20f5000090032000200780041
:100860000090a0000200e0000200350000202400fb
:1008700000007100000c78008080eb002d00370034
:100880000100260001006100810f500008003a00bd
:1008900038009000808f5100050039000800780072
:1008a000300007008080eb000000e00021003a00eb
:1008b00000c020001800600017003a00600220000d
:1008c00008004000a8049000808f540012003a00f5
:1008d00000202000260307008000780020049800f4
:1008e0000000e00005003a0029049800490498003f
:1008f0000900e80030049800060037001860a000e6
:10090000400498000020b00030049800410c98008a
:10091000510c98004d0307002800900050049800e7
:10092000380090006004980000002600180c700049
:100930008000eb00010078004f04be0000000600bc
:100940000200e0000500320090cf100004003200e9
:100950000000e8000201e900fbff3a000000eb00a4
:1009600000000600889fbe00000478000000e00040
:100970000f003a006044b8000800d00021a3200016
:10098000608078000000e00004003200f5ff0700fe
:100990000000e00001003d008084eb000804e80056
:1009a00009007800e70f540028003c00f2ff3700f0
:1009b00010d8a30024003200a00490004000900052
:1009c000808f54000b003100090150003840900026
:1009d0000000fb0089007800050907000000e00026
:1009e000110034008084440048009000808f54003f
:1009f000f5ff390028009000400498009800780026
:100a000000c020000080600002003200a8049000b6
:100a100001003700b804900001e8a300090032008b
:100a20006904980008003700a8009000410498006d
:100a300061049800510c98001890a0000080eb0011
:100a400002003700590c98000000eb004f04be0074
:100a500000000600010878000000060090cf10009a
:100a6000050032001004e00001003a00000005001b
:100a7000d0cf1000fbff3a00000006000003b100d9
:100a8000030035009000b10001003c00100005009b
:100a9000000005000400fa00889fbe008a9fbe0087
:100aa0008c1f780000047800010678007008900020
:100ab000f8009000010050008808900001005000ec
:100ac0009808900001005000a80890000100500014
:100ad000b808900001005000c8089000810550003f
:100ae0000002220090bf9f0000032300a0bf9f00d0
:100af000081090000028a30018003a000b00e00046
:100b0000160034000b0578008a047800e20f5500c7
:100b100001003600290020000900e0000c0034002c
:100b200058009000c801900009017800ee8057003d
:100b300003000100500498008080eb000000e000fa
:100b40009c0032006808900009004000600c98008a
:100b5000090555004240a900ebff3c0078019000d8
:100b60000200e0000c00340058009000c801900022
:100b70008c00780003000100500498008080eb0096
:100b80000000e0008b00320068089000f800900040
:100b900001004000600c9800080890000000e00090
:100ba00016003400000578008a047800e20f550032
:100bb00001003600290020000900e0000c0034008c
:100bc00058009000c801900009017800ec8057009f
:100bd00003000100500498008080eb000000e0005a
:100be000740032006808900009004000600c980012
:100bf000090555004240a900ebff3c001809900090
:100c00000200e0000c003400e80090005800900062
:100c1000c801900003000100500498008080eb00a0
:100c20000000e0006300320068089000980890001f
:100c300001004000600c9800280890000000e000cf
:100c400016003400000578008a047800e20f550091
:100c500001003600290020000900e0000c003400eb
:100c600058009000c801900009017800ec805700fe
:100c700003000100500498008080eb000000e000b9
:100c80004c0032006808900009004000600c980099
:100c9000090555004240a900ebff3c0038099000cf
:100ca0000200e0000e003400e800900018089000f8
:100cb0008080400058009000c801900003000100af
:100cc000500498008080eb000000e0003900320002
:100cd00068089000b808900001004000600c98007f
:100ce000480890000000e00016003400000578007d
:100cf0008a047800e20f5500010036002900200028
:100d00000900e0000c00340058009000c801900079
:100d100009017800ec80570003000100500498009e
:100d20008080eb000000e0002200320068089000a4
:100d300009004000600c9800090555004240a900d8
:100d4000ebff3c00081090000028a30018003200c0
:100d50000b00e000160034000b0578008a047800d0
:100d6000e20f550001003600290020000900e000d4
:100d70000c00340058009000c80190000901780070
:100d8000ee80570003000100500498008080eb00c3
:100d90000000e000070032006808900009004000f1
:100da000600c9800090555004240a900ebff3c008b
:100db0008000eb00010078004f0678004f05be0070
:100dc0004f04be000080fa0000000600889fbe00ad
:100dd0008a1f78000004780001027800024578003c
:100de000830478000200fb00cf80de005002b100d7
:100df0000180b10032052000820f5000e08f5800c2
:100e000095013e00006001008d013700920137001e
:100e100091013700900137008f0137008e013700b4
:100e20008d0137008c0137008b0137008a013700b4
:100e300089013700880137008701370086013700b4
:100e400085013700840137008301370082013700b4
:100e500081013700800137007f0137007e013700b4
:100e60007d0137007c0137007b0137007a013700b4
:100e70007901370078013700ed003700760137003f
:100e80007501370074013700e9003700e8003700ca
:100e9000e7003700700137006f0137006e0137003f
:100ea0006d0137006c0137006b0137006a013700b4
:100eb00069013700680137006701370066013700b4
:100ec0004b013700640137006301370062013700ce
:100ed00061013700800037005f0137005e01370095
:100ee0005d0137005c0137005b0137005a013700b4
:100ef0005901370058013700cd003700560137003f
:100f0000150037001c003700c9003700c800370043
:100f1000c700370050013700170037004e01370077
:100f20004d0137004c0137004b013700ec00370012
:100f3000690037001f0137004701370046013700bd
:100f40002b013700440137006300370042013700ae
:100f500041013700600037006e0144001200780044
:100f6000808141009480e900010a78000009e800ce
:100f70009149780041013700a8609000c0c6b300d5
:100f800080cf50000a003a0094007800648050003e
:100f9000000a78001000be004f89de00cf91de000d
:100fa0000002be00020378008203780015003700bb
:100fb00010c7b30080cf500002003a00140178003f
:100fc0000400370014017800a0c6b30080cf5000a1
:100fd00005003a0068005100000a78003002be00a7
:100fe0002003be00070037000280e900000a7800f5
:100ff0001000780000027800cfa2de000503780020
:1010000086037800049cbe000694be00a860900091
:1010100080c6b30080cf50000f00320020c6b3005e
:1010200080cf500006003a00184078000000fb0016
:10103000cf80de0001017800820178000a003700cd
:1010400040c7b30080cf500003003200664040002c
:1010500080cf500006003a0018007800cf80de00f4
:101060000101780082017800009cbe000294be005d
:101070003800be002801be00e00f5000e08f58008d
:10108000e00f5900e08f590004003d006e0144005c
:1010900092007800d0c2b3000c0037000810900016
:1010a0000018a300040032006e0144009200780092
:1010b000b0c2b300050037000008a300570032009b
:1010c0006e0144009200780000c2b30080f4780002
:1010d0000109e80051003700a8609000c0c6b300c5
:1010e00080cf500006003a009400780064805000e1
:1010f000000a78001002be006033b8001500370007
:1011000010c7b30080cf500002003a0014017800ed
:101110000400370014017800a0c6b30080cf50004f
:1011200005003a0068005100000a78003002be0055
:101130002003be00070037000280e900000a7800a3
:101140001000780000027800050020000600200052
:1011500007002000049cbe000694be00a86090001a
:1011600080c6b30080cf50000f00320020c6b3000d
:1011700080cf500006003a00184078000080fb0045
:101180000100200002002000030020000a003700b8
:1011900040c7b30080cf50000300320066404000db
:1011a00080cf500006003a001800780001002000af
:1011b0000200200003002000009cbe000294be003c
:1011c000081090000038a300140032003800be0060
:1011d0002801be00e00f5000e08f5800e00f5900da
:1011e000e08f59000d00320080c7b300804f5500da
:1011f0000300320080c5b300804f550007003a005d
:101200006e0044009000780002c3b30082f47800be
:101210008100e8008af478000108e8007800900076
:1012200000804400600498008a4078006d00370018
:10123000a860900014017800c0c4b30080cf5000b3
:1012400005003a0068005100000a78005001be0015
:101250004000be000400370064005100000a78001e
:101260001000be0069070700009cbe000294be008b
:10127000380090000000e00004003d006e014400d2
:1012800092007800d0c2b3000c0037000810900024
:101290000018a300040032006e01440092007800a0
:1012a000b0c2b300050037000008a30005003200fb
:1012b0006e0144009200780000c2b30080f4780010
:1012c0000109e80078009000008044006004980064
:1012d0008a40780008007800d901070067003700cd
:1012e000286090008000fb00c0062000808f500026
:1012f000230032000a003c0064005000808f500040
:101300002600320004003c0066005000808f500030
:101310000b00320021003700a00620000500370036
:1013200040072000808f50001c0032001b003c0052
:1013300063005000808f5000070032001700370014
:101340001480e900000a780010007800485c9000e2
:1013500008487800490037001480e900000a780046
:101360001002780068089000cf80de00010178004c
:1013700082017800009abe000292be003f00370052
:101380001480e900000a78001001780068089000d5
:10139000cf80de000089be00380037001480e900ed
:1013a000000a780010007800680c900008087800a7
:1013b000320037001480e900000a7800100078003d
:1013c000cf80de000101780082017800009cbe0021
:1013d0000294be00780090000080440060049800f1
:1013e00081c7b30008007800dc0007002300370045
:1013f0001480e900000a780010007800600498006a
:10140000580990000200e00002003d00850107003d
:10141000090037008000eb0049fd070080007800dc
:101420000000e000030032006800900000805000df
:101430000100370058089000100c98000f0037008a
:101440006e0144009200780050c2b30080f1780031
:101450000109e80009003700ee004400110078009f
:10146000808144000a4278008008e8000a04e00015
:1014700001003a0054c2b300844978000000eb0038
:101480004f0578004f04be0000000600889fbe0094
:1014900080047800c1598000010078000100e0005c
:1014a0000a003a00a1b320003a0be2001c0032000f
:1014b00011007800908f5400140036008080e800fe
:1014c0001100e000faff3a00150037001100e000bb
:1014d0000600320011017800928f54000b00360094
:1014e0008280e8001100e000faff3a001001780065
:1014f000a1b32000d0598000820f500008003200b4
:1015000011007800908f540002003e000100780026
:10151000150037008080e800910f1100f8ff3a00b5
:10152000e8598000890f5400010031000904780057
:101530000800780099030700000178000000e0002f
:1015400005003a000000eb00890f5400060032004d
:101550000804d100f3ff3700081978000200780072
:1015600095030700cbff37004f04be0000000600c4
:10157000881f7800630440000800a1000001eb0010
:10158000800f540022003600e30f540001003e009b
:101590004800200008007800bcff070080007800a9
:1015a0000001eb000000e00019003200100178009b
:1015b0009201780064805100880f500003003100d0
:1015c00012009000800878000700370008004100f2
:1015d0008008780012029000140098001100780032
:1015e0000888510008097800910078000100e000a7
:1015f00004003200110090008180e8000000e0004b
:1016000001003a008000eb00c15988000281e80027
:10161000020078004f04780000000600881f780060
:10162000880020000800d00021a3200060807800fe
:101630000000e000010032000a0007000804e90091
:10164000f8ff3700e0b0200094033700424be2007f
:1016500003003a00fbff070020c0b30042ebb700d5
:1016600000000600889fbe0000047800bdfc070053
:10167000800478001868a30002003200280090005f
:101680004d0307000000eb00200498003840900054
:101690000004e000050035000000fb000206070022
:1016a0000000e000010032008084eb001810900080
:1016b0000000e00008003200040607000000e0001f
:1016c000010032008084eb00181090003a030700fc
:1016d0000000eb00101498001878a3000e003200f0
:1016e0008000eb000100d00022a320000200400097
:1016f000900f1400060032008100e800e78f5000d0
:10170000f8ff3600080078002b03070010003700b0
:101710000008eb00fbff3700000ceb0000c0eb0003
:101720003044980060022000080040002004980027
:101730004004980050049800400c98006004980001
:10174000500c98007004980076004400000c98003b
:10175000090078004f04be00000006006f02b000d0
:10176000889fbe008a9fbe008c9fbe008e1f78009f
:101770008006780030ae2000b0b79f0080c5b3006f
:1017800080cf50000200320022ad2000b2b79f008f
:1017900083002000c3b79f00f0c6b30080cf500085
:1017a0000a0032006940400080cf5000050032003e
:1017b000a4002000c4b79f0080c5b30080cf5000b4
:1017c00002003a0000012000c0b79f008e012000f7
:1017d0003d04be002d05be0040c6b30080cf5000c2
:1017e000030032006540400080cf50000a003a00fc
:1017f000e00f5400e08f5c00e00f5d00e08f5d00c3
:1018000005003d000800be000a01be001e060700dc
:101810000205be000004be00e00f5400e08f5c0033
:10182000e00f5d00e08f5d0003003a005d0890006e
:101830000000e0000c0032007e012000cfb09700d5
:1018400001027800cfa2de0005037800860378004d
:101850000800be000a01be00a10607003fb29700c3
:1018600064407800d0e79f004fb09700cf80de0043
:101870000101780082017800d0b79f00e1b79f0096
:10188000f2b79f0083bf9f000203be000002be00ac
:101890000800be000a01be008a060700809ebe0046
:1018a0008296be00e00f5000e08f5800e00f590014
:1018b000e08f5900220034000e00e00020003400c8
:1018c0003d00be002d01be005fb29700efb2970051
:1018d0007fb397008fbb9700850607000205be0007
:1018e0000004be000e07e900e1fc2f008f804000dd
:1018f000010647005fb29700efb297007fb39700f1
:101900008fbb97000800be000a01be001507070044
:101910001d0010003fb19700624e7800889ebe0007
:101920008a96be00e00f5400e08f5c00e00f5d007f
:10193000e08f5d00020034000e00e000e0ff3c009c
:10194000cfb19700e88f510010003a000d109000c1
:101950000038a3000d003200f70f570006003e00cc
:10196000e4fc2f000e024200e4c07f0000c3b3007d
:1019700080cf5000050032000e07e90000c3b3001d
:10198000e1fc2f008e80400080f07f00780117007e
:10199000920e98006d009000e3fc2f008f814100b3
:1019a0008e804100e5fa07001d0e90005d08900052
:1019b000800f560006003d000c005000800e98007d
:1019c0000d1090000040a100801698000f00370015
:1019d0000000e0000d003d000d109000740060005c
:1019e000f00f500009003a007d089000fd009000c3
:1019f000010050008d089000010050000c075000bd
:101a00004240a900010034008e0e98004f07780074
:101a10004f06be004f05be004f04be006f02b1006e
:101a200000000600800078001004e0000200320090
:101a30005104e000feff3a00008050000000060064
:101a4000ef04b000889fbe008a9fbe008c9fbe003e
:101a50008e1f7800c0af9f00a1df9f0060fa2f00ab
:101a60000f004000e0af9f00cfaa97005503be00d3
:101a70004502be0084af9f0095af9f00a6af9f00b8
:101a8000b7af9f0010c6b30080cf500016003200e1
:101a900010c4b30080cf5000130032004fab97004a
:101aa000560890000000e00003003d0060002000a8
:101ab000500b98000c0037000000e0000a003a00cc
:101ac00070c6b300afdb970080cf53000300320035
:101ad00070c4b30080cf530003003a001000200010
:101ae000cfa89700d0089800cfa89700e2fc2f005d
:101af000028047007602070080017800e20f500064
:101b000014003a00cfa99700e300900030002000b5
:101b10009009980010c6b3002fda9700804f52004a
:101b20000a00320064404000804f5200070032003b
:101b30000040e800804f520004003200c2b4200090
:101b40000040e800804f520017003a0002b5200024
:101b5000150037000000e00018003400cfaa9700fd
:101b6000e500900030002000900a980010c6b300f5
:101b70002fdb9700804f53000a0032006440400082
:101b8000804f5300070032000040e800804f5300b0
:101b90000400320042b520000040e800804f5300ae
:101ba00001003a0082b52000b258780002007800a7
:101bb000b058780090487800f201370014c6b3009e
:101bc000afdb970084cf53000300320010c4b30092
:101bd00080cf530010003a004fa89700ec0040005f
:101be0001101780000c3b300005978008208e800b2
:101bf00080c7b300afd8970084cf500001003200f7
:101c000080c5b300004978004fa99700720090008a
:101c10000080e800700198000300e00003003a0033
:101c20008006eb00fda79f00d001370011c6b3006e
:101c3000afd9970081cf51000300320010c4b30028
:101c400080cf5100ad003a00ceb520002fda9700ca
:101c5000814f520001003200deb62000cfaa97006b
:101c6000550890008006e8000000e00001003d00fb
:101c70001d0220000d06e8004fab97003604be00a1
:101c80002605be006022b8006033b8000fa8970098
:101c90009fa897002fa99700bfa997005606070095
:101ca0000000e00001003d000bf0a20088af9f00a3
:101cb00099af9f00aaaf9f00bbaf9f007fa0970086
:101cc00064005000f0a79f00efab9700805beb0033
:101cd000e7af9f003f003700c20120000300200053
:101ce00001fd2f0001804700270207000faa97007f
:101cf0009faa97002fab9700bfab9700f4af9f0050
:101d000085b79f0096b79f00a7b79f000400be004d
:101d10000601be003d0607000004be000005be002f
:101d2000670656004240a9000c0034006306070015
:101d30000002be000203be007fa897008fb097008c
:101d40001fb19700afb197005f06070080af9f00fb
:101d500091af9f00a2af9f00b3af9f00efaa970083
:101d6000e7824200e5af9f0070002000e00f5400c2
:101d7000e08f5c000d003400600020006fab970026
:101d80006f636500e6af9f00cc5bdd004455de006d
:101d90000a857300c4ddde00e00f5500e08f5d00b2
:101da000020034000000e900f4ff3b000000e900fd
:101db00005003300efa897008060eb00e1af9f00c3
:101dc0000000e900fbff3b006fa99700670141009d
:101dd000e2af9f000c00e000090034006022b80070
:101de0006033b8000fa897009fa897002fa997000d
:101df000bfa99700360607000000e000b6ff3c00d0
:101e0000efa9970064fa2f000f02420004805100ee
:101e10000006e90075fa2f0085824700e5af9f00b4
:101e20008d0f560001003d008c0678000d00e0008b
:101e30002b0035008c8f560005003d006fab9700de
:101e400066c07e00f2c0b300e74f500001003c00c6
:101e50000041eb008d00e900efab970067c0780010
:101e6000824f500006003a008d06e9008100e9002b
:101e7000efa9970063c07800824f5000faff32004c
:101e8000ef4f510004003a006faa970064c0780039
:101e90000040e80000f278000100e00007003d008b
:101ea000efaa97008502e900e5af9f008d06e800e4
:101eb0007fa0970064004000f0a79f008d00e9001c
:101ec000070033006fab970066c078000000fb008e
:101ed0006e40780000f378008100e900f9ff3b00d4
:101ee000cfab9700570890000000e0001f013d00b5
:101ef0000d00e900d00b98001c0137000fac9700d3
:101f00009fac97002fad9700bfad97006022b8003f
:101f10006033b8000800be000a01be00b605070025
:101f20000000e00005003d000bf0a20088af9f001c
:101f300099af9f00aaaf9f00bbaf9f007fa0970003
:101f4000725927000280b900026a2800130020009d
:101f50000c040700e4005000f1a79f001d003b00a7
:101f600063801000c1ff2f00010460000800ea0038
:101f7000f0a79f008004eb000800e0004700340059
:101f80000808a3000e0032006848b800a2a820008c
:101f9000020040003002be002003be000fa89700e0
:101fa0009fa897002fa99700bfa99700cd0507000c
:101fb00080af9f0091af9f00a2af9f00b3af9f0083
:101fc0000884d1008904e8000800e000ecff3c0030
:101fd000320037000100e000300034006022b80019
:101fe0000600200007ff2300b4b79f00c5b79f007d
:101ff000d6b79f00e7b79f00c0ff2f0000806000aa
:10200000f0a79f00000478008004eb001600340065
:102010000808a300100032006848b800a5a82000f6
:10202000050040003002be002003be003fb0970014
:10203000cfb097005fb19700efb19700a9050700f7
:102040000002be000203be00b4b79f00c5b79f00e8
:10205000d6b79f00e7b79f000884d1008904e80045
:102060000800e000eaff3c003fb29700cfb29700c3
:102070005fb39700efb397000fa897009fa8970052
:102080002fa99700bfa997000b06070080af9f00fc
:1020900091af9f00a2af9f00b3af9f004fab9700df
:1020a000d608900060c6b300afdb970080cf530026
:1020b000040032006687400060c4b30080cf530044
:1020c00003003a007fa09700008040006a074000ac
:1020d000f30f5700010034003e01200000c3b3009d
:1020e000efa8970080587800e1af9f003a003700d2
:1020f0000800be000a01be00440507000006be003d
:10210000f0b79f0081bf9f00680757004240a900b9
:102110000e003400690507000002be000203be0085
:102120000800be000a01be00670507006022b80073
:1021300046782d00771924006a05070080af9f00bc
:1021400091af9f00a2af9f00b3af9f00efa9970090
:10215000e8814100e3af9f0088002000e00f5600b7
:10216000e08f5e001100340078002000a200200003
:10217000030020007fb097008fb897007801070018
:102180006faa970005c3b30005624100e4af9f004a
:10219000f0b79f0081bf9f00e00f5000e08f580014
:1021a000020034000804e900f0ff3b000804e900e5
:1021b0000600330000c3b300efab970080637800e4
:1021c000e7af9f000804e900faff3b006fa8970003
:1021d00068004000e0af9f000e00e0000b003400fc
:1021e0000fac97009fac97002fad9700bfad970045
:1021f0006022b8006033b8000800be000a01be00cb
:10220000330507000000e000b9ff3c00efa897008d
:1022100062fa2f000f014100028050000007e90020
:1022200073fa2f0083814700e3af9f007fa09700e0
:1022300067004000f0a79f0001c3b30093cf1000d8
:102240000a003a000e07e9007fa097000000e900ad
:10225000f0a79f006faa97000402e800e4af9f0078
:1022600014427800814f5200f6ff3200cfaa970047
:10227000d508900060c6b3002fdb9700804f530055
:102280000300320060c4b300804f530004003a00e2
:102290007fa09700008040008006e8000a00370019
:1022a0008001eb0050c6b300afdb970080cf530036
:1022b0000300320050c4b30080cf530001003a0045
:1022c00013002000838640008d0f570001003d0061
:1022d0008e0678000d00e000240035008e8f560039
:1022e00006003d006fa89700e0c07e0092c3b300d7
:1022f00040c3b30080cf500001003c0002c3b300d4
:102300008d00e900efa9970063c07800824f50006c
:1023100006003a008d06e9008100e9006faa9700e7
:1023200064c07800824f5000faff320090c3b300bf
:10233000804f510004003a00efaa970065c0780072
:102340000040e80080f278000100e00007003d0056
:102350006fab97000603e900e6af9f008d06e8002b
:102360007fa097000000e800f0a79f007fa29700e1
:102370008d0178006fa99700afd897004fa89700fc
:102380000e0107004f0778004f06be004f05be0044
:102390004f04be00ef04b100000006000000e000a2
:1023a00003003400d2020700e10f400001003a00b0
:1023b0000000eb00000006000000e00036003200e4
:1023c0000081e90012027800e30f5200320036006b
:1023d0000408a30030003a00d15980000100e00059
:1023e00002003200810f5100030031000108780023
:1023f000d25988001d00370081017800110090003b
:102400000000e00008003200820f5000060031009a
:1024100080017800100090000000e000020032000f
:10242000820f5000faff39009300780001804100cc
:10243000800f510018003900820f500003003a004d
:102440008489400003017800080037009300900061
:102450000100e0000300320004004100808f5000c2
:102460000d0039001101980092019800920090002f
:102470000100e000080032009201780003004100f2
:10248000810f500004003a00382bef001089410002
:102490001000900010019800000006000001780074
:1024a000000020000000e000080032000000800072
:1024b0000000e000050032000000e9000000880094
:1024c0000000d0000100800002b07800000006008b
:1024d000889fbe00800478000104780031009000dd
:1024e0000000d0004501de00f07f2000800f510089
:1024f00010003a00800ceb00310090006f0060008b
:1025000008003a00210090000000e00005003a00b9
:10251000110090000000e00002003a001100e0000d
:1025200002003200200020001500370010002000bb
:10253000130037000200e00005003c0001007800b5
:10254000cf010700000178000000e0000a003c0015
:1025500038009000f10028000100600001fe230017
:10256000010070003004980020c02f00800c410052
:102570000080eb0002003700800ceb000000eb0055
:102580004f04be0000000600881f78008a9fbe002e
:10259000000478000205be00300190000200d00067
:1025a000c500de00f07f2000808f50000c003a0054
:1025b0006f00610008003a00280090000000e00071
:1025c00005003a00180090000000e00002003a0008
:1025d0001800e0001c003200200020005d003700e1
:1025e0000100e00006003a0008007800a40107009e
:1025f000800078000000eb000100e00055003c0086
:102600006108b9000a0540008b854800e07f200082
:10261000800f5500e08f5d000d0034003800900001
:102620006022b8000600200007ff2f000000e00035
:10263000030035006022b8000600200007ff2700d5
:10264000049cbe000694be0010002000410037002c
:10265000b8009000e00f5500e08f5d0005003400e9
:10266000f000280000806000c450dd000100700010
:102670003600370000002800808260006f80600014
:102680000040a0003004980061055500e0855d0021
:10269000c0fc2f00f1ff2f00800f5500818f5d00df
:1026a00006003d00350498000000eb00200498006f
:1026b00010049800000ceb00260037000a02780096
:1026c000f00f45000b003c0018009000000c780053
:1026d0002800900010049800380090002004980012
:1026e0000000eb003004980070024200f00f42003e
:1026f000f5ff34000402ea001200320018017800ed
:102700000411de00f0011200180090008300dd00cb
:10271000010c71000400de00280190008310dd0030
:1027200001007000100498000411de0038009000d1
:102730008301dd0003017100220498000400de0023
:1027400030049800380090000500700030049800b4
:102750000080eb004f05be004f047800000006002b
:102760000400fa00889fbe008a9fbe008c9fbe00b6
:1027700080bf9f0091bf9f000206be0001020700bc
:102780000001be000004be000c00be00a40407004f
:102790000fb997009fb99700000551008185590036
:1027a0000800be000a01be004f06be004f05be0075
:1027b0004f04be000080fa00000006000a00fa0084
:1027c000889fbe008a9fbe008c9fbe0000047800d8
:1027d00001457800820578008304780004067800bb
:1027e0000300e00002003c00190020006bb820004c
:1027f00060c6b300804f55000e00320060c4b300c5
:10280000804f55000b00320070c6b300804f55005a
:102810000300320070c4b300804f550083003a00bb
:10282000e40f46008100350058089000800f5600e4
:102830007e003d000c06e80060c6b300804f5500e6
:102840001000320060c4b300804f55000d0032000c
:10285000081090000038a30004003a0058089000c7
:10286000808f540001003d00590c980058089000da
:102870000c005000500c980002003b000000eb00e0
:10288000500c98000c00e00027003c00f2014400ce
:10289000130178006800900001c3b3000170790053
:1028a0000201e80082097800580890000000e0006a
:1028b00003003c00081090000038a3000400320020
:1028c000e8009000e0c2b300807079008209e8005f
:1028d0000c00ea00d8089000808f500001003d00f5
:1028e0000106ea000c00ea00200c98000c80400071
:1028f000500c9800890f500001003d0080047800c2
:10290000680090009808900001004000390c980081
:10291000090178008b00780008f70700580890003c
:10292000090050001a003700e800900018089000d5
:102930008c8f540018003d00008040000901780091
:102940008b007800fdf60700180890000901400090
:10295000120c980009005600200c980058089000ae
:102960000000e00003003c00081090000038a300c5
:1029700006003200e8009000e0c2b30080707900e9
:10298000380890000000e800300c980058089000cb
:10299000400c9800a3003700008040000c01780034
:1029a0008b007800e5f60700180890000c00400046
:1029b000100c98008c845400580890000000e0002f
:1029c00003003c00081090000038a300060032000d
:1029d000f20144009300780068019000e0c2b30067
:1029e00000f178008109e80058089000890f500034
:1029f00001003d0080047800680090009808900075
:102a0000010040008c80450009017800cbf60700ea
:102a10001808900009004000100c98005808900019
:102a200009005000200c98007e00370070c6b300eb
:102a3000804f55000300320070c4b300804f550032
:102a400014003a0058089000808f540004003d00a4
:102a5000081090000038a30001003a00590c9800bb
:102a6000580890000000e900500c980002003b005c
:102a70000000eb00500c980051c6b30070c6b300c4
:102a8000804f55000100320051c4b3000145780069
:102a90000900370010c6b300804f550002003a000d
:102aa0000ac7b3000400370010c4b300804f5500bc
:102ab00001003a000ac5b300f20144001301780096
:102ac000680090003b7079000201e80082097800fc
:102ad000580890000000e00003003c00081090003f
:102ae0000038a30004003200e8009000e0c2b30008
:102af000807079008209e800580890000000e0002a
:102b0000100034008904e900890f500001003d00e5
:102b10008004780068009000980890000100400050
:102b2000090178008b00780084f6070018089000ef
:102b300009004000100c980058089000090050004f
:102b4000200c9800e8009000180890008085400054
:102b50008a5d78008b06e8000c00e0000400350078
:102b6000b0c2b300804d78008d05780004003700b6
:102b7000d0c2b300804d78008d0578000c06ea00c5
:102b80008004eb000c00e00009003400a1002000ec
:102b90000c0078008d0007007681540001f17f0061
:102ba000000678008904e8000000e000f7ff3c0020
:102bb000e18f540009003c0050c6b300804f55001f
:102bc0000300320050c4b300804f550003003a00a8
:102bd00000c3b300805e78008d0578000900e00036
:102be00002003a0000c3b300805d78000900e000f5
:102bf000070034008904e900f680540061c07f00ba
:102c000002c3b300825d40000900e000f9ff3c0010
:102c10006800900098089000010040000080550076
:102c2000300c98000810900074006000f00f500005
:102c30000e003a00780090009808900001004000d3
:102c4000a808900001004000b80890000100400072
:102c5000c80890008100400078089000808f5000e4
:102c600002003d0001005000000c98004f06be001d
:102c70004f05be004f04be000080fa0000000600b1
:102c8000000278003000900001002800010360007d
:102c9000150020006f0060003002980008003a0024
:102ca000240090000000e00005003a0014009000ad
:102cb0000000e00002003a001400e0003e00320094
:102cc000340090000000e0000b003a002400900067
:102cd0003002980014009000200298001400780040
:102ce00010029800000aeb00f082520034009000bd
:102cf0000000e000f5ff320034009000ef0f5000bc
:102d000014003e008001d000a40090004f08de00b7
:102d100080817100330298008100d000140190007e
:102d20004f10de0080807000210298000201d00068
:102d3000940078004f08de00000171001202980034
:102d4000010ad0008502e90003007800ef8f5100ee
:102d5000ecff3600b4019000ff8f510013003600e5
:102d60001401d10014009000cf00dd00010a7100b1
:102d70000000d100a40090004f09dd0002007000a7
:102d8000100298008100d1004f18dd008080700093
:102d9000210298000300d100300298008502e8006b
:102da00080017800ff0f5000edff3e0034009000de
:102db0006f00600030029800340090000600700040
:102dc000300298000500780000000600010178003c
:102dd00000027800110009000200d8000002fd0086
:102de0000491b900820250000400be0000000600f9
:102df0000a00fa0000027800c3202000e52020002d
:102e00000721200046212000e20f50001b003e0059
:102e1000405a8000e10f500004003200632120007e
:102e200085212000a7212000e621200013409000ea
:102e30000078a30002003a00000beb0013f0a000a2
:102e4000154090000028a30001003a0015a0a00042
:102e5000820178000200e00010003200154090006e
:102e60000008a300fdff32003100fb00800b78005a
:102e70008301e900f9ff3a00080037003000200024
:102e8000b0bf9f00c4bf9f00d1bf9f00e2bf9f00a3
:102e90006a80570000c0da006fb99700020078001e
:102ea0000080fa00000006000a00fa00110020006d
:102eb000b1bf9f00c0bf9f006a80570000c0da000a
:102ec0004fb897000080fa00000006000a00fa00e0
:102ed00051002000b1bf9f00c0bf9f006a80570013
:102ee00000c0da005fb897000080fa00000006001a
:102ef000889fbe00800478004a0be20005003a007b
:102f00000000eb00100007008080eb000000e000f4
:102f10000a003500585a8000880078000900e00057
:102f20000600320009004400070007008080eb0023
:102f30000000e00001003500880078000100780002
:102f40004f04be0000000600800078000001eb0086
:102f50000000e00003003a0080b82000505a8800ca
:102f600006003700c0d72000808f500002003e00ce
:102f7000515a8800010037000081eb000200780000
:102f800000000600839f68000100e00002003d0091
:102f900060001000e08018000300e00002003d0027
:102fa00060011100e0811900080007004f00e000f7
:102fb00002003b0060001000e080180000000600e6
:102fc000020007000400be00000006006022b800f6
:102fd000060220000000d0008180d2000482d200ce
:102fe0008582d2000000a0000202520083825a00b3
:102ff00003003b000202420083824a000000a1005d
:103000000603e900f3ff3a000000060081037800a0
:10301000890207000001be006000b8000478a30028
:1030200013003a006220e10015003e000d00390057
:103030008301d1000281d3008180d3008301d100bc
:103040000281d3008180d3008301d1000281d300ab
:103050008180d3000538b000c42add00f300b2003f
:103060008381720007f0a70003f0a00000000600b3
:10307000f3ff2700f2ff2f006110b900fbff3700bc
:1030800003ff2700f7ff370060001000e080180002
:1030900060011900e081190000000600881f780017
:1030a000000478005001be004000be000000420055
:1030b00081804a0002014b0083814b00009cbe00ce
:1030c0000294be00dc0007000300310048009000bd
:1030d0000000e800400498004f047800000006005b
:1030e000889fbe00000478008004eb005001be0001
:1030f0004000be00d0000700010031001900200090
:10310000040050008580580006015900878159004d
:10311000009cbe000294be004800900009005000d0
:10312000400498004f04be00000006001200fa00a0
:10313000889fbe008a9fbe008c1f78000205be00db
:103140000004be00f4b79f0085bf9f0096bf9f009c
:10315000a7bf9f000000eb00e0b79f00d0b79f0023
:10316000c0b79f00b0b79f00a0b79f000006eb005c
:103170005fb197006fb097008000d0000000e000c2
:1031800015003d00e1b79f00010078000200e0005b
:1031900001003d000000a000ac00070001003d0060
:1031a0000000a000af00070001003d000000a000eb
:1031b000b200070001003d000000a00081000700f0
:1031c00001003d000000a000b20007007c80570015
:1031d000b2ff070014003700e1b79f00010078003c
:1031e0000200e00001003d000000a0009700070081
:1031f00001003d000000a0009a00070001003d0012
:103200000000a0009d00070001003d000000a0009c
:103210006c00070001003d000000a0009d000700b9
:103220007c805700aeff07006fb097000000e00001
:103230000700350010002000010020006011b800d8
:1032400008047000898470000a0571008b85710084
:103250000c06e800f0032000800f5600c4ff340085
:103260006fb097000000e00006003d007fb29700bd
:103270008fba97001fbb9700afbb97007c805700a9
:1032800086ff07000802be000a03be006fa8970071
:103290000000e00004003a002fb29700bfb2970090
:1032a0004fb39700dfb397000400be000601be00d5
:1032b0004f0678004f05be004f04be000080fa00a4
:1032c00000000600881f780018002000881f780082
:1032d00096ff07008f87e9004f0478000000060082
:1032e000801feb0091ff07008f87e90000000600b8
:1032f0000800fa00889fbe008a9fbe008c1f7800dd
:103300006e00070005003d00430007003000070085
:103310000c003d00330007000b003700e00f5200a7
:10332000e08f5a00e00f5b00e08f5b0006003d007d
:103330000400be000601be0053ff07000205be00e8
:103340000004be001c0020002c000700ddff070069
:103350000c00e000010032004bff07004f06780030
:103360004f05be004f04be000080fa0000000600ba
:103370000800fa00889fbe008a9fbe008c1f78005c
:103380004e00070002003d001c0020002200070044
:103390000f00070001003d001200070017000700a2
:1033a000cfff07000c00e0000100320036ff0700ed
:1033b0004f0678004f05be004f04be000080fa00a3
:1033c0000000060090b79f000100d00080b79f006a
:1033d000e00f5400e08f5c00e00f5d00e08f5d00c7
:1033e000000006000800be000a01be0026ff07001c
:1033f0000205be000004be00000006000802be0078
:103400000a03be005fb09700efb097007fb197004e
:103410008fb99700000006001bff0700010007009e
:1034200000000600b0b79f00c1b79f00d2b79f0051
:10343000e3b79f00000006000400e1000588e100fa
:103440000690e1000798e10000000600c0b79f0069
:103450000200d000b0b79f00afb097000100e000bd
:1034600000000600b0b79f000100d000a0b79f0089
:103470009fb097000100e00000000600a0b79f0089
:103480000100d00090b79f008fb097000100e000ce
:103490000000060080b79f000804d0008984d20095
:1034a0000a85d2008b85d2005fb29700efb29700f9
:1034b0007fb397008fbb970000000600d9ff07007d
:1034c0000605be000404be000006eb00e00f50003d
:1034d000e08f5800e00f5900e08f5900000006000f
:1034e000889fbe008a9fbe008c9fbe000404b80067
:1034f0000506b8008904460060854e000606b8003f
:103500000a054600e0854e000706b8008b05460018
:10351000040eb800890446000a854e00050eb80066
:103520000a0546008b854e00060eb8008b05460046
:103530000416b8000a0546008b854e000516b80033
:103540008b054600041eb8008b0546000800be002f
:103550000a01be004f06be004f05be004f04be006c
:10356000000006000800fa00889fbe008a9fbe0087
:10357000170007000605be000404be00e00f52005d
:10358000e08f5a00e00f5b00e08f5b0008003d0019
:103590000400be000601be00bbfe07000205be001f
:1035a0000004be000f000700b7fe07000800070078
:1035b0000802be000a03be000a000700c8ff070099
:1035c0004f05be004f04be000080fa000000060058
:1035d000e0b79f00f1b79f0082bf9f0093bf9f009d
:1035e000000006006fb09700ffb097000fb997007a
:1035f0009fb99700000006008f1fd100230107002c
:103600008f87e9000000e000000006001400fa00c7
:10361000889fbe008a9fbe008c9fbe000004be0033
:103620000205be00680047000a90be000890be0078
:103630003f0107000070a7000bf0a10030432000fd
:103640009e02900080825200b0fe2f000028e10010
:1036500011003d00b0fc2f000028e10015003400ef
:103660001e0990008e0890007e0090000501b000b9
:103670000201d1008180d3000080d3008502e800e0
:10368000fbff3a000b00e00064013b00600010000b
:10369000e080180061013700f0ff2f00f1ff2700e4
:1036a0000b00e0005d013b0001002800000020004d
:1036b0005a0137006000b800580137004f89de001a
:1036c000820178005a01370007f0a2008f0137000d
:1036d000809feb00ed0007008f87e9000000e0000d
:1036e000000006002800fa00889fbe008a9fbe00e6
:1036f0008c9fbe0003866b00340107000028a300e6
:1037000064003a000128a30067003a000008a30003
:1037100062003a000108a30065003a001e00900014
:10372000be08900081064000ed3fb100f4805700d4
:10373000ee019000111ab8008e099000311bb800fc
:103740009e099000311cb800511db800f485570047
:1037500046000700fe0190003a0007008b85e80054
:103760003e0007008e09900040000700ee01900027
:10377000340007008b85e800380007008e099000b0
:10378000400007009e0990001b18b8008904400003
:103790000a854800fe019000340007008b85e80090
:1037a00038000700ee019000300007008e099000fd
:1037b0001b18b800890440000a8548000a98a30035
:1037c00008003a000402420085824a0006034b00ca
:1037d00087834b0008044c0089844c000a054d0087
:1037e0008d06e90084827200850273004c3add0088
:1037f000850272000100320015002000443ade000c
:103800001400b2004538de00cb45dd000b0070002f
:10381000c540de00cb4ddd008b8070004549de00e9
:10382000cb55dd000b017100c551de000d037800a2
:10383000b301070003f0a1000cf0a70003f0a00003
:10384000f60037001b18b8008502400006834800c8
:10385000e0834b0060044c00070037001b18b800e1
:103860000603400087834800faff37001b18b800a2
:103870008703400008844800e0844c0060054d0048
:10388000000006001b18b8000804400089844800a6
:10389000faff37000108a300dd003a005800be001f
:1038a0005801be00e3ff37000008a300d8003a002b
:1038b00009047800f9ff37002800fa00889fbe004d
:1038c0008a9fbe008c9fbe0003866b00bf0007006e
:1038d0006400e100440032006408e1004a00320064
:1038e0006100e100460032006108e1004900320059
:1038f000ec0647006000b8003d02be003d03be007c
:10390000f48657006011b8003d04be003d05be00be
:103910007d0320000b0037000000a0008d06e900a9
:10392000130032000402420085824a0006034b0065
:1039300087834b000000400081804800020149005d
:10394000838149000802520089825a000a035b0001
:103950008b835b00f0ff3b000802420089824a0033
:103960000a034b008b834b008d06e900edff3a0004
:103970008482720086827200f707b200878272002a
:1039800001003200150020001e0490003e0b900044
:1039900006035400e63fb0000368a30007003200ae
:1039a0000000a7000500a0008301d1000281d30020
:1039b0008180d3000080d3000603e8008301d1009a
:1039c0000281d3008180d3000080d3000002eb008d
:1039d0000482d2004a01070003f0a1000cf0a70006
:1039e00003f0a0008d003700640247006408e10086
:1039f000870032003400be003401be00f6ff3700fd
:103a00006108e100820032006011b8006000b80077
:103a1000f1ff370003ff270002002000fbff370003
:103a2000020ab900001bb9000200b8008100420080
:103a30008100430000000600c70ade00f107b20063
:103a4000f50fb20008003200e1cf42000200320060
:103a50000170a00024000500810f700001003200f9
:103a60000408050044000500810f700002003a00c0
:103a7000140005008502e9000000400081c04800f4
:103a8000fcff3b000170a00024000500889fbe00e1
:103a90008a9fbe008c9fbe000404be000605be00c7
:103aa000809fbe00829fbe0041010700040678008f
:103ab0000800be000a01be003d0107008406780030
:103ac0004f03be004f02be008d4f76007fb09700bf
:103ad00013003300f0ff2f008b8f6b0006003b00bc
:103ae0000d0666000c00a7000a00370007f0a600cc
:103af000100020000a003700880f5200898f5a00fa
:103b00008a0f5b008b8f5b000300390010002000e0
:103b100001003e000000200007f0a7000000ea00be
:103b20004f06be004f05be004f04be000000060059
:103b3000800078005002be005003be004439de0011
:103b4000f700b200f37f200003016100090032009a
:103b50000218e10016003a0085017200830173002b
:103b6000838173000008200015003a004000200007
:103b70001300370085017200830173008381730095
:103b800005003a0004a8be0006a8be0010002000f0
:103b90000b0037000201e9000402420085824a005e
:103ba00006034b0087834b000748a300f9ff320050
:103bb0000740a00004a8be0006a8be002000200008
:103bc00080009800920098000000060068044700fa
:103bd0000294be000094be00fc0447008694be0020
:103be0008494be0009007800d1ff07000800780027
:103bf000cfff070099007800814f70000b003b0059
:103c00000800be00fc0007004f00b10003003700b1
:103c1000f3ff2700f2ff2f006110b9004f06be002e
:103c20004f05be004f04be000080fa0000000600f1
:103c3000889fbe00830478000300e0002c0035005c
:103c400003003c0000827000040271002600320074
:103c500036432000c50020008383cf000a003900ce
:103c60000541b1008283cf00070039000541b10052
:103c70008183cf00040039000541b1008083cf006b
:103c8000010039000541b10085c353006022b8002e
:103c9000120032000a003b00848272006102600060
:103ca0008301d1000281d3008180d3000080d30042
:103cb0000603e8008743e800f7ff3a0007003700f3
:103cc00000004000818048000201490083814900d2
:103cd0000603e9008743e900f9ff3a00880007007e
:103ce00009f0a70003f0a0004f04be00000006008a
:103cf00060001000e080180060011900e0811900e8
:103d0000d3ff3b00033e2c00f7ff37002800fa00ea
:103d1000889fbe008a9fbe008c9fbe000706780069
:103d2000878669000c003b00030478008704780054
:103d300008f0a10009f0a100840f5000858f580001
:103d4000860f5900890f5c00030033000cf0a200bd
:103d500001003a000cf0a1009cff07006400e100a4
:103d60005f003200780147006408e1006100320022
:103d70006c014700748557003200be001201be007e
:103d80003a04be001a05be001e039000be0a900051
:103d90008503530006003d000004fd008104fd0082
:103da0000205fd008305fd008703ea000503780096
:103db0000df8a3000400320060041400e0841c002d
:103dc00060051d00e0851d006022b8007d03200015
:103dd0000d38e1008006eb000b0039004433dd00b4
:103de000f300b2008301730039003700848272004f
:103df0000d027800e10664008b85d1000a85d300ae
:103e00008984d3000884d3008703e900f7ff3b00cf
:103e100008004000898048000a0149008b81490060
:103e200004003b0060001000e080180060011900f1
:103e3000e08119000358a300090032008d8272004e
:103e400084827200610260008301d1000281d3008c
:103e50008180d3000080d3000603e8001b003700f8
:103e60000348a30017003a000600e00017003400e2
:103e70000603e9000d00a30000004800818048000f
:103e800002014900838149000348a3000f003a0062
:103e90000600e000090034000603e90000004000cd
:103ea00081804800020149008381490001003a00f5
:103eb0000003eb000348a300f5ff32006022b800c6
:103ec0000200370084827200618266000c000700e5
:103ed00003f0a1000cf0a70003f0a0004fff370093
:103ee000640147006408e10002003a000df8a300f5
:103ef00047ff3a003200be001201be0047ff370004
:103f00001800200057002000080453000d003d0059
:103f10000600200097fc2f000740e1001e0034003f
:103f200084827200610260008301d1000281d300ab
:103f30008180d3000080d3000804e800f8ff3a0035
:103f4000470020006104600005047400040464005c
:103f50000d00320061004000e0804800600149002f
:103f6000e081490003b8a500070032000603e8001d
:103f70006538e10004003a008301d1000281d300da
:103f80008180d3000080d300f87f20000830e1005a
:103f900003003500080378006000b8006011b80025
:103fa0004433dd00f300b20083017300000006001b
:103fb00005ff270005826100070032000428e100a8
:103fc00001003200240005000600070001003a004d
:103fd000440005000408050002000700f9ff3a004c
:103fe000140005006f82610081027000850271007b
:103ff0008502720000000600e48240001078a300f1
:1040000007003200640240001178a3003400be00b3
:104010001401be00040032000330a70000000600b7
:104020003500be001501be000330a00000000600f0
:104030000000fa000000eb0050158800f01f280077
:1040400040158800e000200030158800000820009e
:10405000201588000000eb001015880000002800e3
:10406000001588000080fa00000006000200fa0037
:10407000000f78009e0078006f8060003015880087
:10408000a022a800401f2000e7100700a022a900de
:10409000a0c2bf000080fb00610060000000e000e3
:1040a000fbff3200001480000080fa0000000600d0
:1040b0003200f800900188006118e100040032002d
:1040c0007018e10002003200f0ff2f0003003700fb
:1040d0003119ba008301e900fdff3a003200f9000e
:1040e00000000600849fbe004220a9004404240072
:1040f0006110e1000a003200540424007010e10055
:104100000700320064042400f5ff2f000510e100d1
:1041100003003200f0ff2f004f02be000000060037
:104120003200f800203b8800113b8800043b8800e7
:104130000500fc0050052000303b8800a00a20004c
:10414000303b880061e7a80000000000000000008c
:1041500061e7af00feff37000000eb003200f9001e
:104160004f02be0000000600841f78004220a90014
:10417000440024006118e1000600320054002400cd
:104180007018e100030032004f027800f0ff2f00aa
:10419000000006003200f80091018800821f7800bc
:1041a0003019bb008301e900fdff3a00213b880084
:1041b0004f017800123b8800043b88000500fc009a
:1041c00050052000303b8800a00a2000303b8800ca
:1041d00061e7a800000000000000000061e7af00f8
:1041e000feff37000000eb003200f9004f027800bc
:1041f000000006000200fa000000eb00000f78004b
:10420000a00020009e0f100008003c001e00780057
:104210000000d00022972000820040000000eb0048
:10422000800878001e0fe800f5ff3700900020009e
:10423000404c8800007d2000604c88004006200033
:10424000704c88000000eb00804c8800300020009b
:10425000904c88000000eb00504c8800c0122000f9
:10426000a04c880060042000b04c88008002200030
:10427000c04c88000000eb00d04c88000000eb0030
:10428000e04c8800a004220001002000004d8800be
:10429000114d88007008200001002000204d88008a
:1042a000314d88000078200001002000404d88003a
:1042b000514d88008000200001002000604d8800e2
:1042c000714d88008000200001002000804d880092
:1042d000914d880020032000a04d880000f42100ab
:1042e000b04d88001300200022962000010f2f00ff
:1042f000f00720006eff0700104b80000000e80070
:10430000104b880012002000010f2f00f007200042
:1043100074ff070013002000020f2f00f107200098
:104320002096200090ff07000080fa0000000600a1
:104330000400fa000000eb00f04c88000000eb00e5
:10434000000f7800600120009e0f100024003e0046
:10435000510120009e8f100008003e001e007800d2
:104360000000d0002297200082004000f04c800026
:1043700011004000f04c880003003700f04c800032
:104380000000ea00f04c88001e0078000000d00019
:1043900002002f008200400012002000f0072000e1
:1043a00050ff0700100798001e0078000000d000a2
:1043b00001002f00010140001e0078000000d00025
:1043c000219720000100400013002000f107200089
:1043d00065ff0700100798001e0fe800d9ff37009f
:1043e000804c8000e10f500009003a009e09f8005f
:1043f0001e019000821f78001e007800801f780048
:10440000407e2c00801f7800ecef0700e887570003
:104410000080fa00000006000600fa000000eb0031
:10442000200798000000eb00000f780060012000da
:104430009e0f100015003e001e0078000000d00006
:1044400021972000010140001e0078000000d000ec
:1044500003002f008300400013002000f00720001d
:1044600013ff0700100798001e0078000000d0001e
:1044700022972000820040002e0090001100400092
:10448000200798001e0fe800e8ff37001300200007
:1044900022962000010f2f00f007200004ff0700e4
:1044a0002e0090000080fa00000006000400fa00d0
:1044b0000000eb00c04d88000000eb00000f78000a
:1044c000c00020009e0f100024003e00b10020001c
:1044d0009e8f100008003e001e0078000000d000f3
:1044e000029a200082004000c04d80001100400070
:1044f000c04d880003003700c04d80000000ea0076
:10450000c04d88001e0078000000d00002042f007b
:104510008200400012002000f0072000f1fe07009a
:10452000100798001e0078000000d00001042f0042
:10453000010140001e0078000000d000019a200018
:104540000100400013002000f107200006ff0700d3
:10455000100798001e0fe800d9ff3700804c80003c
:10456000e10f500009003a00b809f8001e01900060
:10457000821f78001e007800801f7800d0802c00f9
:10458000801f78008def0700e88757000080fa0051
:10459000000006000600fa000000eb00200798006b
:1045a0000000eb00000f7800c00020009e0f1000fc
:1045b00015003e001e0078000000d000019a200087
:1045c000010140001e0078000000d00003042f000d
:1045d0008300400013002000f0072000b4fe070015
:1045e000100798001e0078000000d000029a2000fa
:1045f000820040002e00900011004000200798002b
:104600001e0fe800e8ff37002e0090000080fa003f
:10461000000006000e00fa00000f78001107980055
:104620009e00900040062000008ab9001e0078001d
:104630006101b9000400be0052fa0700300798007b
:104640004107980042062000030020003e00900031
:10465000ce00900000005100818059005007980062
:10466000610798005e009000ee009000e00f50009f
:10467000e08f580004003c001000200001002000e2
:104680005007980061079800100320009e0f10004b
:10469000150034003e009000ce009000420620003d
:1046a0000202b8000001eb000283b90005017800a6
:1046b00006014100430620000388b90000014100c3
:1046c00082027800007122000100200004004000f6
:1046d000858048005e019000ee01900029fa0700f5
:1046e00020079800020037000000eb002007980028
:1046f0002e0090000080fa00000006000000fa0082
:104700005a0ae20005003a0070832c00c308070033
:104710000000eb00f04a88001e0037005e09e2004e
:1047200005003a0010002000f04a8800e101200056
:10473000f0a42000510e0700e04a800062006000f3
:104740000000e00003003200d0832c00b308070013
:1047500010003700e04a8000640060000000e000c4
:104760000300320030842c00ac0807000900370039
:10477000e04a8000680060000000e00003003200b2
:1047800090842c00a508070002003700f0842c005c
:10479000a20807000080fa00000006000200fa00ec
:1047a000c1498000207520000088b9004108de0062
:1047b00001002000c04a8800c04a80008a07070024
:1047c0000080fa00000006000600fa005a09e20024
:1047d0003f003200624a8000734a8000804a8000b5
:1047e000914a8000800f5100818f590007003400ea
:1047f000604a8000714a8000804a8800914a88009f
:10480000e0152000f05288001b0037005e0ae2002d
:1048100019003a0020032000f0528800804a8000ee
:10482000914a80008180d1000080d3001007980059
:10483000210798001e009000ae009000e00f50008d
:10484000e08f580004003a006000b800804a8800f9
:10485000914a880008003700804a8000914a800011
:104860001e019000ae0190000200500083805800ad
:10487000804a8800914a880050852c00670807000c
:10488000814a8000804d8000000ab800814a800083
:10489000904d80000088b9000501780000014100ba
:1048a000814d8000904a80000088b90000014100dd
:1048b0008202780040a8de00cf80de00000f780082
:1048c000710720001e0078008d09070005003700e1
:1048d00090852c00510807006000b800804a8800cd
:1048e000914a88000080fa00000006000000fa00eb
:1048f0005a09e2001800320090002000dbfd07009a
:10490000cf80de00024d80000202b800124d800010
:104910000283b9000501780006014100034d8000c3
:104920000198b900000141008202780040a8de0031
:10493000cf80de00e049880010862c003708070091
:1049400011002000e04980006d09070030862c002e
:10495000320807000200370050862c002f0807009d
:104960000080fa00000006000000fa004005200068
:104970000308070041072000104a80006009070073
:1049800000022000fe07070040002000fc0707008f
:1049900030042000fa0707000080fa00000006003b
:1049a0000000fa00a14d8000c0f62000b30d070002
:1049b00061060700004b2000e0528800d4c2bf000f
:1049c0000080fb0061006000e10f50001e003a0013
:1049d0000040eb004e060700e0528000c2122000ab
:1049e000110009000280d800801f7800d0862c00ba
:1049f000801f78000091200051ee0700e4875700e7
:104a0000009120000508070000c4b300400607001d
:104a100000882c00010807005c0ae200e7ff3a006a
:104a2000a04d80008000d000e0252100930d0700fc
:104a3000d4c2bf000080fb0061006000e10f5000a5
:104a4000fbff3200ddff37005c0ae2000c003a0099
:104a500037fe0700804c8000e10f500004003a0050
:104a600010892c00801f780054ee07008f87e90022
:104a700020002000890e0700cfa2a900ffff370009
:104a80000080fa00000006000000fa00e7c2bf0044
:104a90000080fb004700de000080fb000000e0001b
:104aa00004003200ca82a900e04a80000020a00071
:104ab000e04a8800114a8000b04c8000808f50008e
:104ac00004003400ca82a900e04a80000030a0003f
:104ad000e04a8800a14a8000a04c8000808f5000ee
:104ae00008003400b14a8000a04c8000808f500044
:104af00004003400ca82a900e04a80000010a0002f
:104b0000e04a88005c09e200020032000000eb008d
:104b1000204988000080fa00000006000000fa002a
:104b20000000eb00e04a88000000eb00f04a88003b
:104b3000caa2a90040012000580e0700caa2a8007e
:104b40000080fa00000006000200fa00fa050700e3
:104b5000e08b2c00b107070000c4b300ec05070090
:104b6000f08c2c00ad070700680f07000004e00080
:104b700011003200750f0700004f7800a1002000df
:104b8000f0a420003d0d07001e407800500f0700e4
:104b900000c4b300de050700008e2c009f0707004d
:104ba0001e80fb0076070700a08e2c009b070700e5
:104bb0001e40780078070700d4c2bf000080fb00c9
:104bc00061006000e10f5000e7ff3a000080fa004a
:104bd000000006000200fa000000eb00000f780061
:104be000900020009e0f100008003c001e0078007e
:104bf0000000d00022a72000820040000000eb004f
:104c0000800878001e0fe800f5ff37004001200003
:104c1000405488000000eb00305488000080fa0007
:104c2000000006000200fa00860ae20029003200b5
:104c30006c09e200150032000000eb00000f780064
:104c4000900020009e0f10000c003c001e00780019
:104c50000000d00021a720000100400010007800d3
:104c6000801f7800f08e2c00801f7800d3ed0700a5
:104c7000e48757001e0fe800f1ff3700308f2c004b
:104c8000801f7800cded07008f87e90090538000ea
:104c9000e40f50000e003c0090002000000f780050
:104ca0001e00e000080034001e0078000000d00064
:104cb00021a72000010040001000e00002003a009f
:104cc0001e0fe900f6ff37001e007800404c8800f8
:104cd000c0ff07000080fa00000006000200fa0092
:104ce000b0002000e1fc0700000f78001000200059
:104cf000704b88000080fa00000006000400fa00f3
:104d0000b0002000d9fc070010079800a000200088
:104d1000000f78001e00e00009003400a17c2c0088
:104d20001e0078000000d000810040001e009000ae
:104d3000910f500002003e001e0fe900f5ff370002
:104d40001e007800404c88000080fa000000060039
:104d50000400fa00404c80000000d00021972000a1
:104d60000100400010007800000f78001e0078005d
:104d7000e10f5000110032009e007800e18f5000da
:104d800004003c001e0078000000e0000800320033
:104d9000120037009e007800e28f50000a003200b7
:104da0001e007800e30f50000a0032000b003700ad
:104db000cae2a800cac2a80008003700cae2a900d7
:104dc000cac2a80005003700cae2a800cac2a900ea
:104dd00002003700cae2a900cac2a900414c800003
:104de000110798001e009000e40f500029003200c7
:104df0009e009000e48f50000d003c001e009000cb
:104e0000e10f50000e0032009e009000e18f500034
:104e10002e0034001e009000e20f50000f00320000
:104e20009e009000e38f50001300320027003700ef
:104e30001e009000e60f50001d00340023003700d4
:104e4000e9a2a800e982a900e9c2a900c4e2a90078
:104e5000c4c2a900e802a90022003700e9a2a90003
:104e6000e982a800e9c2a900c4e2a900c4c2a9005d
:104e7000e802a9001b003700e9a2a900e982a90005
:104e8000e9c2a800c4e2a900c4c2a900e802a900be
:104e900014003700e9a2a900e982a900e9c2a9002b
:104ea000c4e2a800c4c2a900e802a9000d003700ae
:104eb000e9a2a900e982a900e9c2a900c4e2a90007
:104ec000c4c2a800e802a90006003700e9a2a900b0
:104ed000e982a900e9c2a900c4e2a900c4c2a900ec
:104ee000e802a8000080fa00000006000200fa00b4
:104ef0009c09e20024003200504c8000000f780032
:104f00001e007800e10f50000d0032001e007800f6
:104f1000e10f500004003c001e0078000000e0009b
:104f200005003200180037001e007800e20f500024
:104f300014003200140037003aff07001200370057
:104f40004a0ae20010003a00b609e2000e00320000
:104f5000b04d800050528800504c8000e10f50004e
:104f600009003a00260be20002003a00a0002000ef
:104f7000404c8800430f07000000eb0030598800c8
:104f8000010037005dff07000080fa000000060006
:104f90000000fa00e000200034fc0700cf80de00b3
:104fa000f0498800014a8800f0498000014a8000e9
:104fb00002fa20000202b8000001eb000283b900ef
:104fc000050178000601410003fa20000388b900ba
:104fd00000014100820278004028de00010020002c
:104fe000104a8800d000200020fc0700c04988003b
:104ff000c00020001dfc0700d0498800c149800086
:10500000c04980000088b900204a8800314a8800e1
:10501000d1498000d04980000088b900404a88000a
:10502000514a8800224a8000334a8000404a80006a
:10503000514a80000000510081805900604a880078
:10504000714a8800a04a8000b04a8800d149800097
:10505000c04980006ffd0700a04a88000080fa0068
:10506000000006000000fa00c04c8000ea0040008a
:10507000104a8000810f500003003400e842a8006d
:10508000e862a80011003700c04c8000e500400035
:10509000104a8000810f500003003400e842a8004d
:1050a000e862a90009003700114a8000c04c800066
:1050b000808f500003003400e842a900e862a80095
:1050c00002003700e842a900e862a9000080fa0067
:1050d000000006002600fa00f0f32f0000168800fa
:1050e0000000eb001016880080e0270030168800d2
:1050f0000000eb0040168800e001240060168800e4
:105100000000eb0070168800100020009016880048
:105110000000eb00a0168800c0c72f00f016880022
:105120000000eb000017880000002800201788000e
:105130000000eb0030178800e862a800cfa2a800aa
:1051400040442500a0048800260b0700c0cc2100a5
:1051500060488800ea0a07007f040700c8040700c7
:1051600075040700608f2c002c06070040742c008b
:105170002a06070000c4b3006504070020902c0035
:1051800026060700b50d0700a9fb070030912c008b
:10519000220607000000eb005049880080bb200079
:1051a000e0528800d4c2bf000080fb0061006000b4
:1051b000e10f500019003a005c0ae200f9ff3a00e2
:1051c000c1122000e0252100ac0b070000c4b30091
:1051d0004f040700c0912c001006070010002000ab
:1051e00050498800d4c2bf000080fb00610060000d
:1051f000e10f5000fbff32000040eb0044040700c9
:10520000d0922c000506070000c4b300400407003c
:10521000e0932c0001060700e2ff3700ddfc0700e9
:10522000300798007cfc070040079800804c800005
:10523000e10f500009003a006209f8004e009000aa
:10524000801f7800be009000811f7800f0942c0031
:10525000801f780059ec0700e88757003e00900057
:105260000000e00003003a004e0090000000e00063
:10527000080032009907070060992c00801f780011
:105280004eec07008f87e900dafb070087fc070078
:1052900027fc0700604c8000f80a0700704c800073
:1052a000f00a07000000eb00204988000000eb0036
:1052b00030498800404c8000e90f50000200340063
:1052c00090002000404c8800a04d80008000d0005d
:1052d000f0a42000690b0700caa2a900e842a800b8
:1052e000e862a900007d20006c0c07001204070092
:1052f000caa2a800e842a900e862a9002a09e200bf
:1053000001003200b508070000000000cec2bf0057
:105310000080fb004400de000080fb0061006000b4
:105320000000e00012003a000040eb00f803070024
:10533000709c2c00b905070000c4b300f4030700fb
:10534000809d2c00b5050700c3c2bf000080fb0094
:105350004400de000080fb00610060000000e0000f
:10536000eaff3a00a3fb070050fc0700f0fb070030
:105370005afe0700904c8000460d0700804c8000cc
:10538000e10f500027003a00909e2c00801f78000b
:105390000aec07008f87e90040742c00801f78001a
:1053a00006ec07008f87e900b09f2c00801f780073
:1053b00002ec07008f87e900a0742c00801f7800a2
:1053c000feeb07008f87e900f09f2c00801f78001c
:1053d000faeb07008f87e9000c09f80070a22c0097
:1053e000801f7800f5eb0700e4875700904c8000a1
:1053f000e30f50000b003200914c80008000200031
:105400000008b80052752c0000004100801f780091
:105410009209f800f0a32c00801f7800e7eb07004a
:10542000e6875700c3c2bf000080fb004500de00d6
:105430000080fb00610060000000e00001003a0015
:10544000c1fd07000000eb00404988000000eb00b0
:1054500020498800a0002000004b88008001eb005c
:10546000630f9800cac2bf000080fb000000d1009b
:105470000080fb00610060000000e00002003a00d4
:1054800010002000600f9800ce58900061c06000ae
:105490000041d000a12c200091407800d0cfb30073
:1054a00000c0600002407000cae2b700c8c2bf007e
:1054b0000080fb004300de000080fb006100600014
:1054c0000000e0000300320010002000d04a8800f5
:1054d000020037000000eb00d04a880083fe07007e
:1054e000abfe070068fd0700c3c2bf000080fb00e1
:1054f0004500de000080fb00610060000000e0006d
:1055000051003a00803e2000e05288002409e20069
:1055100007003a0030498000e40f500004003a00d0
:10552000a14d8000c0f62000d40a07000d0037000e
:1055300020498000e10f500007003a0040498000f8
:10554000e70f500004003a00a14d8000c0f6200093
:10555000ca0a070003003700a14d8000a07f210088
:10556000c60a070000000000c3c2bf000080fb00a5
:105570004500de000080fb00610060000000e000ec
:1055800008003a005c0ae200f7ff3a00a14d8000f3
:10559000a00020000088b90080007800c0f620003c
:1055a000b60a07005c0ae20011003a0020498000b8
:1055b0000000e8002049880020498000e10f5000e9
:1055c000020034000000eb002049880000000000c9
:1055d000c3c2bf000080fb004500de000080fb006e
:1055e000610060000000e000f9ff320013003700a6
:1055f0002409e20009003a00304980000000e80078
:105600003049880030498000e40f50000b0034001e
:105610000000eb0030498800080037004049800056
:105620000000e8004049880040498000e70f500032
:10563000020034000000eb0040498800e109070047
:1056400040062000950b0700cec2bf000080fb0083
:105650004400de000080fb00610060000000e0000c
:1056600019003a009a09e20002003a005c09e200df
:1056700006003200a14d8000c0f620007f0a07001e
:105680000000eb00d04c880005003700a14d8000e1
:10569000a07f2100790a070010002000d04c88006c
:1056a000400620007d0b0700cec2bf000080fb003b
:1056b0004400de000080fb00610060000000e000ac
:1056c000f9ff320015fd0700c3c2bf000080fb00d8
:1056d0004400de000080fb00610060000000e0008c
:1056e00026003a007dfd07006e09e2001700320037
:1056f0009c09e2000d003a0010002000e04c8800f8
:1057000034fd07000000eb0050528800424c80003e
:10571000024b8800a0002000404c8800a14d800072
:10572000a07f2100550a07000b0037000000eb00a6
:10573000e04c8800034b8000434c8800a14d800062
:10574000c0f620004d0a070003003700a14d80007d
:10575000c0f62000490a0700400620004f0b070052
:10576000c3c2bf000080fb004400de000080fb00dd
:10577000610060000000e000f9ff3200cec2bf000f
:105780000080fb000000d1000080fb006100600091
:105790000000e00025003a009c09e2000800320009
:1057a0000000eb00e04c8800004b8000404c88007b
:1057b000a14d8000c0f62000300a0700120037001b
:1057c000404c80000000e800404c8800404c8000c5
:1057d000e90f50000200340090002000404c880087
:1057e000404c8000e90f500004003a00a14d8000b9
:1057f000f0a42000210a070003003700a14d80001b
:10580000a07f21001d0a070040062000230b07008f
:10581000cec2bf000080fb000000d1000080fb0072
:10582000610060000000e000f9ff3200cec2bf005e
:105830000080fb004300de000080fb006100600090
:105840000000e00024003a009c09e2000800320059
:105850000000eb00e04c8800014b8000414c8800c8
:10586000a14d8000c0f62000040a07001100370097
:10587000404c80000000e900404c88008809e200ac
:1058800002003c0010002000404c8800404c80008a
:10589000e10f500004003a00a14d8000c0f6200046
:1058a000f609070003003700a14d8000a07f21000a
:1058b000f209070040062000f80a0700cec2bf0028
:1058c0000080fb004300de000080fb006100600000
:1058d0000000e000f9ff32001dfd0700d04a800003
:1058e000e10f500010003a00d04c8000e10f500052
:1058f0000b003a005c09e20007003a00404c8000cf
:10590000ea0f5000040032008809e2000200320071
:10591000ca82a80005003700ca82a9000300370028
:10592000ca82a90001003700ca82a900cdfd070084
:105930000040eb0076020700224980002217980001
:10594000ae1190000300e000030032002e10900022
:10595000e10f5000f700320090fb07003149800052
:10596000710f98007e099000e20f51002100320073
:10597000fe099000e28f510007003c007e08900075
:105980000000e0000a003200fe089000e18f5000a5
:105990000b003200060037007e099000e30f510033
:1059a0004b003200fe099000e48f51004c003200a1
:1059b00070c0b3008802070083fb07004b0037006c
:1059c00070c0b3008402070090a62c0013040700e7
:1059d0005409e20003003a00d0a62c000f0407008f
:1059e0004200370021002000a04a80004405070043
:1059f0003e003700a00020009cf90700cf80de00a9
:105a000092498000a3498000020140008381480040
:105a100092498800a3498800f05980000000e800fe
:105a2000f0598800f0598000ef0f50002f0034002b
:105a30000000eb00f059880090498000a1498000e7
:105a4000cc09dd004400de0000807100c488de0067
:105a5000224d80000202b800324d80000283b9005e
:105a60000501780006014100234d80000198b9002e
:105a70000001410082027800340f9800450f980021
:105a80006000b80090498800a14988003e08900055
:105a9000ce0890004809dd004800de0000007100db
:105aa000c808de008049880070c0b3004a020700c1
:105ab00030a72c00d9030700210020008049800076
:105ac0000f05070050a72c00d4030700070037007c
:105ad00070c0b3004002070084fb070003003700da
:105ae00070c0b3003c0207009ffb070000c4b30076
:105af00007020700404c80000000d00023972000e0
:105b00000300400010007800001798000e1090006d
:105b1000e10f5000110032008e109000e18f500014
:105b200004003c000e1190000200e000080032006a
:105b3000120037008e119000e28f51000a003200ef
:105b40000e109000e30f50000a0032000b003700e7
:105b500070a72c00b103070008003700a0a72c0095
:105b6000ae03070005003700d0a72c00ab030700e9
:105b70000200370000a82c00a80307005c09e2001f
:105b800019003a009a09e20002003a0030a82c00fd
:105b9000a2030700d04c8000e10f500013003a0030
:105ba0005a09e2000d0032005c09e20008003a00e8
:105bb000404c8000ea0f5000050032008809e200e6
:105bc0000300320090a82c00940307000700370060
:105bd000f0a82c00910307000400370050a92c0006
:105be0008e03070001003700c4fa07009c09e20099
:105bf00003003200b0a92c00880307000200370020
:105c0000f0a92c008503070052792c00414c80003c
:105c1000300020000008b800000041001000fb0028
:105c20005703070052792c00414c800030002000bf
:105c30000008b800000041000000e8001000fb0070
:105c40004f03070052792c00414c800030002000a7
:105c50000008b800000041000080e8001000fb00d0
:105c60004703070030aa2c006c0307005508070003
:105c7000200798002e0090000000e000080034008b
:105c8000404c80000000d00021972000010040001f
:105c90001008e800a14d8000a07f2100f708070050
:105ca0002e0090000000e00008003d00404c800005
:105cb0000000d00022972000020040001008e900f8
:105cc000a14d8000a07f2100ec080700404c80001f
:105cd0000000d00023972000030040001000e000e7
:105ce00006003d00404c80000000d00022972000bc
:105cf000820040000000eb0080087800404c8000eb
:105d00000000d00023972000030040003100200055
:105d1000908f10003c013400404c80000000d00007
:105d20002297200082004000300020008008780088
:105d30003501370043498000131798001e1090006a
:105d4000e30f5000900032009e109000e38f50004f
:105d50000a003c001e119000e10f51003d0032008e
:105d60009e119000e18f51005f003c001e109000da
:105d70000000e0000e003200830037009e1090000b
:105d8000e58f5000c20032001e119000e40f510058
:105d90009d0034009e119000e68f5100dd0032001e
:105da0001e109000e70f5000fa0032007600370016
:105db0000040eb005601070070aa2c0017030700f3
:105dc00000c4b30052010700fe070700514c8000d9
:105dd00000804000504c88008a09e20002003d002b
:105de0000000eb00504c8800504c8000e20f500047
:105df0000200340020002000504c880080ab2c00b2
:105e000006030700504c8000e10f500002003a00ea
:105e10000000eb00804c88008a09e20002003a0092
:105e200020ac2c00fd020700504c8000e10f500018
:105e300002003a00a0ac2c00f8020700504c800091
:105e4000e20f5000f0003a0020ad2c00f3020700f2
:105e5000ed0037000040eb002d010700a0ad2c0045
:105e6000ee02070000c4b30029010700504c800077
:105e7000e10f500003003a000000eb00804c880066
:105e800004003700cf070700814c800000804000ed
:105e9000804c88009009e20002003d000000eb0009
:105ea000804c8800804c8000e10f500002003400dc
:105eb00010002000804c8800b0ae2c00d7020700f4
:105ec0009009e20002003a0040af2c00d302070024
:105ed000804c8000e10f5000cb003a00d0af2c0086
:105ee000ce020700c80037000040eb0008010700a1
:105ef00060b02c00c902070000c4b3000401070011
:105f0000b0070700500f98005e0890000000e00006
:105f10000f003200904c8000de089000010040002d
:105f2000904c88009209e20002003d000000eb0066
:105f3000904c8800904c8000e70f50000200340025
:105f400070002000904c8800904c8000510a07009f
:105f5000914c8000800020000008b80052752c0091
:105f600000004100801f780070b12c00801f780075
:105f700000912000f2e80700e4875700009120001c
:105f8000a6020700a00037000040eb00e000070079
:105f900040b22c00a102070000c4b300dc000700df
:105fa0008807070080007800704c800001004000e6
:105fb000704c8800714c8000c0442000808f5000dd
:105fc00002003400c0442000704c88008e09e200ba
:105fd00002003d000000eb00704c88008e09f800c4
:105fe00050b32c00801f780000912000d4e80700f7
:105ff000e48757000091200088020700704c800061
:1060000098070700800037000040eb00c000070041
:1060100070b42c008102070000c4b300bc0007006c
:106020006807070080007800200320000088b9007e
:10603000624c800000004100604c8800614c800090
:10604000c0da2000808f500002003400c0da200047
:10605000604c88008c09e20002003d000000eb006b
:10606000604c88008c09f80080b52c00801f7800f7
:1060700000912000b2e80700e4875700009120005b
:1060800066020700604c80007c0707005e00370056
:106090000040eb009e00070080b62c005f02070066
:1060a00000c4b3009a00070046070700800078008c
:1060b000a00020000088b900a24c80000000410030
:1060c000a04c8800a14c800080bb2000808f500035
:1060d0000200340080bb2000a04c8800a14c80004e
:1060e00030062000808f500002003c004006200057
:1060f000a04c880090b72c00480207002100200027
:10610000a04c80007e03070020b82c00430207004b
:106110003d0037000040eb007d00070070b82c0008
:106120003e02070000c4b3007900070025070700fe
:1061300080007800b04c800001004000b04c880026
:10614000b14c800040062000808f500002003400d7
:1061500040062000b04c8800b14c800010032000a5
:10616000808f500002003c0020032000b04c8800cb
:106170009609f80080b92c00801f7800009120005b
:106180006fe80700e4875700009120002302070012
:106190001d0037000040eb005d00070090ba2c00a6
:1061a0001e02070000c4b3005900070005070700de
:1061b00080007800c04c800001004000c04c880086
:1061c000c14c800040062000808f50000200340047
:1061d00040062000c04c88009809e20002003d0003
:1061e0000000eb00c04c88009809f800a0bb2c0010
:1061f000801f78000091200051e80700e4875700d5
:106200000091200005020700804c80000000e000a3
:1062100002003a00ce0a070001003700da03070047
:10622000d4c2bf000080fb0061006000e10f50009d
:106230008afc3a00daf9070088fc37000200fa000d
:10624000004f78000900fc00b1168000f00f20001c
:10625000008160001e80fb00c800dd0000f02f0000
:106260000080600000007100b0168800100020005f
:106270006d080700d6a2a800100020006a080700d9
:10628000d6a2a90010002000670807000080fa00cd
:10629000000006000200fa0000002800000f78004d
:1062a0000400fc009116800000f02f0000807000b8
:1062b00090168800d6c2a800d6e2a9001e00e00011
:1062c0000a003d001000200057080700d6a2a800d1
:1062d0002000200054080700a116800000f02f00c5
:1062e000008f6000d6a2a900f4ff3700d6c2a90033
:1062f000d6e2a8000400fc0090168000f10f2000f8
:1063000001006000901688000080fa00000006007e
:106310000200fa00004f7800deff0700d6e2a90075
:1063200000c8b3001e407000c4ff0700d6e2a800fa
:106330000080fa00000006000000fa00d5ff070008
:10634000d6e2a90010c0b300bcff0700d6e2a80047
:106350000080fa00000006000000fa00d6e2a90062
:10636000d6c2a900f00020004c08070080c3b3008b
:10637000b2ff0700500020004808070080c3b300a8
:10638000aeff0700100020004408070080c3b300e0
:10639000aaff07001000200040080700c0c0b3009b
:1063a000a6ff0700100020003c08070010c0b30043
:1063b000a2ff0700200020003808070060c0b300db
:1063c0009eff07001000200034080700d6e2a80056
:1063d0000080fa00000006000200fa00004f78007a
:1063e000acff07001e40780094ff07000080fa0011
:1063f000000006000200fa00004f780011479800e4
:10640000a4ff0700d6e2a900f0c3b3001e4f60004e
:1064100000c4b3001e40700088ff0700d6e2a80049
:106420009cff07001e40900084ff0700c2ff07008a
:106430000080fa00000006000400fa00004f780017
:10644000114798000040eb0020479800ae409000b4
:106450001e40900080cf500007003d008dff0700d8
:106460001e40780075ff07002e4090000040e800b5
:1064700020479800f5ff37000080fa000000060072
:106480000000fa0083ff0700d6e2a90000c4b300b1
:106490006aff0700d6e2a80011c0b3000040eb007d
:1064a000e5ff070051c0b30000c1b300e2ff0700e1
:1064b00021c0b3000040eb00dfff070011c0b300b4
:1064c0000040eb00dcff070051c0b30040c1b30047
:1064d000d9ff070021c0b3000040eb00d6ff070042
:1064e00011c0b3000040eb00d3ff070051c0b30060
:1064f00050c1b300d0ff070021c0b3000040eb0043
:10650000cdff070011c0b3000040eb00caff070039
:1065100051c0b30010c0b300c7ff070021c0b300d3
:106520000040eb00c4ff070011c0b300c0c1b300be
:10653000c1ff070011c0b30040c1b300beff070098
:1065400011c0b300c0c1b300bbff070051c0b3000e
:106550000040eb00b8ff070021c0b3000040eb0093
:10656000b5ff070011c0b30000c1b300b2ff0700c0
:1065700011c0b3000040eb00afff070011c0b30033
:1065800000c1b300acff070031c0b3000040eb0016
:10659000a9ff070031c0b3000040eb00a6ff0700d1
:1065a00011c0b30000c1b300a3ff070041c0b30096
:1065b0000040eb00a0ff070021c0b3000040eb004b
:1065c0009dff070031c0b30000c1b3009aff070070
:1065d00031c0b3000040eb0097ff070056ff0700f3
:1065e0000080fa00000006001200fa00000f780098
:1065f000000320009e0f1000020034000003200062
:10660000000f78001e0078006200200011000900d1
:106610000200d800200798001e00780062002000c9
:10662000110009000200d8008000fd00300798002a
:106630000000eb00400798000000eb0010079800f6
:106640001e009000e70f50000e003c00ea004700db
:106650004e0090000081400081bd2c001e00900083
:1066600000804000104978004e0090000000e800d3
:10667000400798001e0090000000e80010079800f6
:10668000efff37000000eb00400798002e0090005d
:106690000000e0000c003400ea0047004e009000cb
:1066a0008080400020c0b300804878004e009000f9
:1066b0000000e800400798002e0090000000e9006c
:1066c00020079800f1ff37003e0090000000e00036
:1066d00007003400ea0047004e00900000814000af
:1066e000c1bc2c003e0090000080400010497800a2
:1066f0000000eb00100798001e009000e70f50000c
:1067000009003c00ea0047001e00900000804000a5
:106710001040780030ff07001e0090000000e800e5
:1067200010079800f4ff37000080fa000000060010
:106730001600fa00000f78001107980000032000ef
:106740009e0f10000200340000032000000f7800ac
:1067500080002000500798001e0078006200200092
:10676000110009000200d800300798001e007800d0
:1067700062002000110009000200d8008000fd0026
:10678000400798001e0090000000e00036003a002c
:106790000000eb00600798003e0090000000e00061
:1067a0000f003400ee0047006e0090008080400033
:1067b00020c0b300804878006e0090000000e80020
:1067c000600798003e0090000000e9003007980044
:1067d0005e0090000000e90050079800eeff3700cf
:1067e0004e0090000000e0000d003400ee00470075
:1067f0006e00900000814000c1bc2c004e00900053
:1068000000804000104978006e0090000000e80011
:10681000600798005e0090000000e90050079800b3
:106820000000eb0020079800ae0090005e00900092
:10683000808f500042003d00ee0047006e00900047
:106840008080400000c2b300804878006e00900055
:106850000000e800600798002e0090000000e800ab
:1068600020079800f0ff37007000200060079800b4
:106870003e0090000000e0000f003400ee004700f2
:106880006e0090008080400020c0b30080487800f7
:106890006e0090000000e900600798003e00900044
:1068a0000000e900300798005e0090000000e90059
:1068b00050079800eeff37004e0090000000e00007
:1068c0000d003400ee0047006e0090000081400093
:1068d00021bd2c004e00900000804000104978003f
:1068e0006e0090000000e900600798005e009000d4
:1068f0000000e900500798000000eb002007980016
:10690000ae0090005e009000808f50000c003d00b3
:10691000ee0047006e0090008080400000c2b3008f
:10692000804878006e0090000000e9006007980041
:106930002e0090000000e80020079800f0ff3700cc
:106940000000eb00200798002e009000e70f500099
:1069500009003c00ee0047002e009000008040003f
:10696000104078009cfe07002e0090000000e80018
:1069700020079800f4ff37000080fa0000000600ae
:106980000200fa00004f78001e40780092fe0700d7
:106990000080fa00000006000200fa00004f7800b4
:1069a0001e407800104798001e80fb004400de0067
:1069b000004f780090c0b3009e4f100003003e00cf
:1069c00000c3b3001e4f40000200370070c3b30085
:1069d0001e4f40001e4078007ffe07001e409000c2
:1069e000004f78001e4078006f4f600090c0b300e9
:1069f0009e4f100003003e0000c3b3001e4f400036
:106a00000200370070c3b3001e4f40001e407800e4
:106a100071fe07000080fa00000006000200fa0084
:106a2000000f78001e0078001004e000070032001c
:106a30009e0078001140780067fe07001e00780075
:106a40000000e800000f7800f6ff37000080fa0031
:106a5000000006000600fa00008fbe0042479800c2
:106a60004e4090000004e0002e003a001e00be00e0
:106a700002a02c00a3b9230042f107000043b0009c
:106a800055fe07001e00be0002a02c00a3b9230083
:106a90003cf1070002a02c000202b800a2b92300ba
:106aa0000283b900050178000601410003a02c0013
:106ab0000388b90000014100820278001e1f120005
:106ac0001e971a00e0c2b30043fe07001e00be007e
:106ad00002102e00535f20002af107000043b0008f
:106ae0003dfe07001e00be0002102e00535f200076
:106af00024f1070002102e000202b800525f2000ad
:106b00000283b900050178000601410003102e0040
:106b10000388b90000014100820278001e1f1200a4
:106b20001e971a004e4090000004e0000a00320058
:106b30001e00be00026829008309200011f1070031
:106b4000e00f5000e08f580003003a0000c2b3008d
:106b500021fe0700060037001e00be000268290063
:106b60008309200007f107000043b0001afe070068
:106b70001e00be00026829008309200001f1070001
:106b8000026829000202b800820920000283b900cd
:106b90000501780006014100036829000388b90057
:106ba00000014100820278001e1f12001e971a0089
:106bb0001e00be0002242400f3002000f1f00700b4
:106bc0000043b00004fe07001e00be0002242400a3
:106bd000f3002000ebf00700022424000202b800ba
:106be000f20020000283b90005017800060141008f
:106bf000032424000388b9000001410082027800c8
:106c00001e1f12001e971a00e0c2b300f2fd07001b
:106c10001e00be00026a280013002000d9f0070001
:106c20000043b000ecfd07001e00be00026a280011
:106c300013002000d3f00700026a28000202b80007
:106c4000120020000283b90005017800060141000e
:106c5000036a28000388b90000014100820278001d
:106c60001e1f12001e971a001e00be000271220095
:106c700003002000c3f007000043b000d6fd07006a
:106c80001e00be000271220003002000bdf00700bc
:106c9000027122000202b8000001eb000283b90079
:106ca0000501780006014100037122000388b90044
:106cb00000014100820278001e1f12001e971a0078
:106cc0001e00be00823e200003002000adf0070041
:106cd0000043b000c0fd07001e00be00823e200041
:106ce00003002000a7f00700823e20000202b80047
:106cf0000001eb000283b9000501780006014100a4
:106d0000833e20000388b900000141008202780020
:106d10001e1f12001e971a00e0c2b300aefd07004e
:106d20001e00be00420620000300200095f0070070
:106d30000043b000a8fd07001e00be004206200070
:106d4000030020008ff00700420620000202b80076
:106d50000001eb000283b900050178000601410043
:106d6000430620000388b900000141008202780038
:106d70001e1f12001e971a001e00be00a200200057
:106d8000030020007ff007000043b00092fd0700e1
:106d90001e00be00a20020000300200079f00700c2
:106da000a20020000202b8000001eb000283b9003b
:106db0000501780006014100a30020000388b90006
:106dc00000014100820278001e1f12001e971a0067
:106dd0004e4090000004e00003003a0001c3b300fd
:106de0001ec040007cfd07000080fa000000060085
:106df0000400fa00008fbe0012c0b3001e00be00e7
:106e000014ff07000080fa00000006000200fa00ec
:106e1000000f78001e00e00002003400b0c2b30092
:106e20006dfd07001e00e00002003a0000c2b30042
:106e300069fd07001e00e00003003d00d0c2b30062
:106e400065fd07001e0fea001e007800823e20004c
:106e5000110009000200d8000043b0005efd0700e9
:106e60001e007800823e2000110009000200d800b8
:106e70008000fd00803e20000088b9001e0f100039
:106e8000e0c2b30054fd07001e0078004206200057
:106e9000110009000200d8000043b0004efd0700b9
:106ea0001e00780042062000110009000200d800f0
:106eb0008000fd00400620000088b9001e0f100071
:106ec0001e007800a2002000110009000200d80076
:106ed0000043b00040fd07001e007800a200200023
:106ee000110009000200d8008000fd00a000200071
:106ef0000088b9001e0f10000080fa000000060094
:106f00000600fa00000f7800110798000000eb005f
:106f100020079800f07022009e0f1000020034003d
:106f2000f0702200000f78009e00900040072000c3
:106f3000808f5000120032001e007800823e200038
:106f4000110009000200d8000000e00005003a002e
:106f500000c2b30020fd07001000200020079800a9
:106f6000090037001e007800823e20001100090051
:106f70000200d8000043b00017fd070002003700f0
:106f800010002000200798001e007800823e20009c
:106f9000110009000200d8008000fd00803e2000a2
:106fa0000088b9001e0f10002e009000e10f500065
:106fb0000c003a001e007800420620001100090073
:106fc0000200d8000000e00006003a001e00900019
:106fd000e20f50000300320000c2b300fefc0700c5
:106fe000060037001e00780042062000110009004c
:106ff0000200d8000043b000f7fc07001e00780034
:1070000042062000110009000200d8008000fd00a7
:10701000400620000088b9001e0f10001e009000de
:10702000e20f500002003a00e0c2b300eafc0700a1
:107030001e007800a2002000110009000200d80004
:107040000043b000e4fc07001e007800a20020000e
:10705000110009000200d8008000fd00a0002000ff
:107060000088b9001e0f10001e009000e10f5000b4
:1070700002003a00e0c2b300d7fc07009e00900077
:1070800070072000808f500003003a0070c5b300e5
:10709000d1fc07000300370001c3b3001ec040004d
:1070a000cdfc07000080fa00000006000200fa0094
:1070b000004f780090c0b3009e4f100002003400d3
:1070c00090c0b300004f780001c3b3001ec0400061
:1070d000c1fc07000080fa00000006000600fa006c
:1070e00000be2c00801f7800b4e407008f87e90001
:1070f0000000eb00000f7800f00f20009e0f100042
:1071000019003c006401470000002f009e00400071
:1071100013002000f0072000e5f307001007980097
:107120001e0078006f0060000000e00006003a00da
:107130001e007800801f780070bf2c00801f780030
:107140009ee40700e48757002e009000801f78001f
:10715000f0bf2c00801f780098e40700e4875700f8
:107160001e8fe800e4ff37001e009000801f7800ab
:1071700040c02c00801f780090e40700e48757008f
:107180000080fa00000006001000fa00df0507008a
:107190000004e0000f013200ec050700204f9800ca
:1071a0002e4890000081fb0003002000f0fb2f0020
:1071b000f1ff2f0002014000838148006207980020
:1071c0007307980060032000010020006e0190000a
:1071d000fe019000800f5100818f5900f2003e00a7
:1071e0006e009000fe009000006001004700370034
:1071f000ed00370057003700eb0037005300370031
:10720000e9003700e8003700e70037002e003700bc
:10721000e5003700e4003700e3003700e200370004
:10722000e1003700e0003700df003700de00370004
:10723000dd003700dc003700db003700da00370004
:10724000d900370054003700d7003700d600370088
:10725000c9003700d4003700d3003700d200370010
:10726000d1003700d0003700cf003700ce00370004
:107270007e003700a1003700cb003700ca0037007e
:10728000ad003700c8003700c7003700c600370020
:10729000c5003700c4003700c3003700c200370004
:1072a000c1003700c0003700bf003700be00370004
:1072b000bd003700bc00370080003700ba0037003f
:1072c000b900370050003700e0c12c00801f780063
:1072d0003ae407008f87e90050c42c00801f780033
:1072e00036e407008f87e90040742c00801f780087
:1072f00032e407008f87e90090c52c00801f7800da
:107300002ee407008f87e900b200370090002000cc
:10731000000f7800e10020009e8f1000ad003c00bf
:107320001e00780051f30700801f78001e017800ce
:10733000821f7800e0c72c00801f78001fe4070040
:10734000e68757001e0fe800f2ff370063ff0700d3
:10735000a0003700c0c82c00801f780017e4070089
:107360008f87e9000000eb00200798001200200042
:10737000010f2f00f00720005af3070064004700b8
:1073800013002000020f2f00f107200076f3070002
:1073900052ff07008f003700b0ca2c00801f780012
:1073a00006e407008f87e900e3fb07002e48900002
:1073b000fb4f500087003200540507000004e00036
:1073c000fdff320061050700204f98002e48900015
:1073d000ed4f500001003a00d7fb07002e48900007
:1073e0000080fb00801f7800e0cb2c00801f78001d
:1073f000f2e30700e48757002e4890000080fb006e
:107400005ffd0700e9ff3700a0cc2c00801f78004b
:10741000eae307008f87e900c7fb07002e489000ca
:10742000fb4f50006b003200a8050700204f98006a
:107430002e489000ed4f500001003a00befb0700bf
:107440002e4890000080fb00801f7800a0cd2c000b
:10745000801f7800d9e30700e48757002e4890008a
:107460000080fb0046fd0700ecff370020ce2c001b
:10747000801f7800d1e307008f87e9000000eb0050
:10748000000f7800f00520009e0f100007003c0060
:10749000a9fb07001e00780053fc07002003200012
:1074a000fe0307001e0fe800f6ff37001705070070
:1074b0000004e000f1ff32004600370030cf2c001e
:1074c000801f7800bde307008f87e9003a050700b9
:1074d000000f780040d22c00801f7800b7e307002f
:1074e0008f87e90034050700100798009e00900080
:1074f0001e007800e10207003600370050d42c004f
:10750000801f7800ade307008f87e9003e00900000
:107510000000e800300798003e00900006020700d7
:10752000a0002000dd030700f80407000004e000cd
:10753000f6ff3200270037006c09e20007003a002e
:1075400010002000604b880030d52c00801f780090
:107550009ae307008f87e9001e0037000000eb0068
:10756000604b880050d62c00801f780093e3070002
:107570008f87e9001700370080d72c00801f780024
:107580008ee307008f87e9000000eb00000f780012
:107590002e0090001e017800110009000200d800a2
:1075a000200798000b0037002e4890000080fb0059
:1075b000801f780060d82c00801f78007fe30700d0
:1075c000e487570030d92c00801f78007be3070048
:1075d0008f87e9000080fa00000006001c00fa0016
:1075e0000000eb00000f780053fb0700804c800088
:1075f000e10f500008003a00a0da2c00801f78004c
:107600006ee307008f87e90070dc2c00801f780094
:107610006ae307008f87e90000000000c8c2bf00ce
:107620000080fb004300de000080fb006100600082
:107630000000e0000300320010002000d04a880063
:10764000020037000000eb00d04a880050f6070027
:107650000df5070025f60700bdf50700d04a8000ac
:10766000e10f50000a003a00d04c8000e10f5000ba
:1076700008003a005c09e20006003a00404c800035
:10768000ea0f500003003200ca82a8000100370050
:10769000ca82a90073f60700d000200073f2070029
:1076a000c0498800c000200070f20700d04988005f
:1076b000c1498000c04980000088b900204a880084
:1076c000314a8800d1498000d04980000088b90043
:1076d000404a8800514a8800224a8000334a80008c
:1076e000404a8000514a80000000510081805900ca
:1076f000604a8800714a8800c3c2bf000080fb0056
:107700004500de000080fb00610060000000e0003a
:1077100013003a001e0fe800500020009e0f1000da
:10772000020034000000eb00000f7800210320006d
:10773000e025210051020700c3c2bf000080fb000a
:107740004500de000080fb00610060000000e000fa
:10775000f9ff32004006200050030700990107009e
:107760009e007800510f98005e099000e20f5100d2
:1077700081003200de099000e28f510007003c00da
:107780005e0890000000e0000d003200de0890006e
:10779000e18f500054003200090037005e0990006c
:1077a000e40f5100d5003200de099000e38f510054
:1077b000a20034005e089000e50f5000eb0032009c
:1077c0000040eb00d2fa0700a000200027f20700db
:1077d000cf80de00224d80000202b800324d8000d2
:1077e0000283b9000501780006014100234d8000a5
:1077f0000198b90000014100820278001407980046
:10780000250798001e009000ae0090004809dd009a
:107810004800de0000007100c808de0080498800d2
:1078200050df2c007dfc07002100200080498000f3
:10783000b3fd0700e0df2c0078fc070000c4b300b4
:10784000b3fa07005f010700cf80de00224d800001
:10785000334d80000201400083814800224d8800a2
:10786000334d8800224d8000334d800030062000cb
:1078700001002000800f5100818f590004003c005e
:107880004006200001002000204d8800314d880076
:10789000224d8000334d8000800c2000010020002c
:1078a000800f5100818f590004003400800c2000ab
:1078b00001002000204d8800314d880066004700ff
:1078c000224d8000334d8000829fbe0021e02c00bd
:1078d000811f78009ae20700e6875700660047009c
:1078e0004efc0700a90037000040eb0088fa0700b3
:1078f000e600470050e12c00801f7800010078006e
:107900008fe207008f87e9006600470043fc07000d
:1079100000c4b3007efa07002a0107008000780047
:10792000a04d800001004000a04d8800b409e20095
:1079300002003d000000eb00a04d8800a14d80003a
:1079400040062000808f50000200340040062000d6
:10795000a04d880066004700b409f80061e22c00e1
:10796000811f780076e20700e48757006600470031
:107970002afc0700850037000040eb0064fa07008e
:1079800070e32c0025fc07008ff3070000c4b30050
:107990005ffa07000b010700cf80de00824d8000f8
:1079a000934d80000201400083814800824d880091
:1079b000934d8800804d8000914d8000e00f500075
:1079c000e08f580003003d006000b800804d880043
:1079d000914d8800824d8000934d80004001200031
:1079e00001002000800f5100818f590004003400f5
:1079f0004001200001002000804d8800914d88004a
:107a0000804d8000914d8000604d8800714d880050
:107a100066004700824d8000934d8000829fbe002b
:107a200021e02c00811f780045e20700e68757001f
:107a300066004700f9fb0700540037000040eb00e8
:107a400033fa070000e42c00f4fb0700a7f307005b
:107a500000c4b3002efa0700da000700cf80de0072
:107a6000024d8000134d80000201400083814800d8
:107a7000024d8800134d8800024d8000134d800098
:107a80007038210001002000800f5100818f5900c3
:107a900004003c008038210001002000004d8800d7
:107aa000114d8800024d8000134d800000712200ae
:107ab00001002000800f5100818f59000400340024
:107ac0000071220001002000004d8800114d880047
:107ad00066004700024d8000134d8000829fbe006b
:107ae000a1e42c00811f780015e20700e68757000b
:107af00066004700c9fb0700240037000040eb0088
:107b000003fa0700b0e52c00c4fb070000c4b30073
:107b1000fff90700ab000700800078004006200056
:107b20000088b900b24d800000004100b04d8800cf
:107b3000b14d800000a62e00808f5000020036005c
:107b400000a62e00b04d880066004700b609f80078
:107b5000c1e62c00811f7800f9e10700e487570097
:107b600066004700adfb0700080037000040eb004f
:107b7000e7f90700e0e72c00a8fb070000c4b3000a
:107b8000e3f90700f0e82c00a4fb070053002000f5
:107b90009e8f110031003a00cec2bf000080fb0072
:107ba0004400de000080fb00610060000000e00097
:107bb0004a003a00803e2000e0528800cec2bf005a
:107bc0000080fb004400de000080fb0061006000dc
:107bd0000000e00041003a005c0ae200f7ff3a00d2
:107be00084f1070031f20700d1f10700a14d8000b8
:107bf000a00020000088b90080007800c0f62000b6
:107c00001e0107000000eb0050498800caf9070078
:107c100000ea2c0081fb0700804c8000e10f50003f
:107c200004003a0010eb2c00801f7800e3e107000d
:107c30008f87e900c05d200018020700cec2bf0098
:107c40000080fb004400de000080fb00610060005b
:107c50000000e000f9ff320027003700cec2bf006d
:107c60000080fb004400de000080fb00610060003b
:107c70000000e00019003a000cf20700a14d80005e
:107c8000c0f62000fd0007000000eb00504988000e
:107c9000a9f90700d0ec2c0060fb0700804c8000a5
:107ca000e10f500004003a00b0ed2c00801f780076
:107cb000c2e107008f87e90000000000cec2bf00cc
:107cc0000080fb004400de000080fb0061006000db
:107cd0000000e000f9ff320007003700d4c2bf0007
:107ce0000080fb0061006000e10f50004bfe3a0095
:107cf0002bf3070049fe37000080fa000000060061
:107d00000000fa00ca42a9000000eb00a059880058
:107d10000000eb00b059880090432000101188004b
:107d200000002800001188008500a9008d00a8002f
:107d30000080fa00000006000200fa00000f780040
:107d4000b05980009e0f10000b00320020c2bf000f
:107d50000080fb000000d1000080fb00610060009b
:107d60000000e000f9ff3a001e00780020118800b2
:107d70001e007800b05988000080fa00000006005c
:107d8000801f78000200fa00ca42a8008500a900fe
:107d900020c2bf000080fb00610060000000e00026
:107da000040032002011800090598800100020004b
:107db000a0598800ca42a9000080fa004f0078004c
:107dc000004006000200fa0080538000000f780097
:107dd0000000eb00805388001e0078000080fa004d
:107de000000006000000fa00400120004054880016
:107df000803e2000705288000000eb00800c88005c
:107e00000000eb00b00c880040062000600c8800e9
:107e100040062000700c8800e0002000800c8800e4
:107e2000007d2000900c8800007d2000a00c8800c0
:107e3000e0002000b00c8800b0cc21007008880061
:107e400013e1a8008ce0a8008c60a90020002000ad
:107e50002008880020032000405288000080fa009b
:107e6000000006000200fa00000f78001e007800f3
:107e7000600c88000080fa00000006000200fa0092
:107e8000000f78001e007800900c88000080fa0037
:107e900000000600809fbe00821f78000800fa00e4
:107ea000a052800030079800be009000e18f500083
:107eb0000c0032003e009000e10f5000060034003c
:107ec000be009000e28f5000200032003e00900083
:107ed000e30f50003b003200d222a8008cc0a90062
:107ee0004c0037008000eb00010f7800d6c2bf00c5
:107ef0000080fb000000d1000080fb0061006000fa
:107f00000000e00002003a0010002000000f78009e
:107f10009e40780061c060000041d000612d2000cb
:107f200091407800d0cfb30000c0600002407000e4
:107f3000d6e2b700600880000000d1006008880029
:107f40000000eb00a0528800320037000000eb0078
:107f500010079800d6c2bf000080fb000000d100cf
:107f60000080fb00610060000000e00002003a00b9
:107f70001100200011079800ae40900061c0600021
:107f80000041d000612d200091407800d0cfb30097
:107f900000c0600002407000d6e2b700d6c2bf0049
:107fa0000080fb000000d1000080fb006100600049
:107fb0000000e0001700320010002000a0528800ee
:107fc000140037000000eb0020079800d6c2bf0065
:107fd0000080fb000000d1000080fb006100600019
:107fe0000000e00002003a00110020002107980084
:107ff000ce40900061c060000041d000612d2000a3
:1080000091407800d0cfb30000c060000240700003
:10801000d6e2b70084c0a9000080fa004f017800c2
:108020004f00be00004006000200fa00000f78007a
:1080300030002000a05288001e00e900600888007f
:10804000600880000000d10030088800d622a90016
:10805000d222a90011e1a80084c0a9008cc0a80008
:108060000080fa00000006000000fa002000200056
:10807000a05288000080fa00000006000400fa0008
:10808000000f780011079800520ae20007003a003a
:108090001e0090000000e000040034001e0090006c
:1080a000805288001e007800dfff07000080fa0081
:1080b000000006000000fa00105280000080fa0064
:1080c000000006003600f800809fbe00829fbe00c0
:1080d000849fbe00869fbe000200fa0084e0a900d3
:1080e00005e1a90000088000105288000000eb00a4
:1080f0000008880005e1a800860ae2001a003a009c
:108100000000eb00000f7800910020009e8f10000f
:1081100009003c00617b2c001e0078000000d000ac
:108120008100400010528000910f50000200360084
:108130001e0fe800f4ff37001e0078000000d0009a
:1081400021a72000010040001008e80040548000f2
:108150000000e90040548800880ae20002003a006a
:108160001000200030548800500ae200060032005f
:10817000805280000000e90080528800500ae2002e
:1081800001003a00b8ff07005c0ae2000300320079
:10819000e05280000000e900e05288007052800048
:1081a0000000e900705288004e0ae20005003a0023
:1081b000803e200070528800704880000000e80077
:1081c00070488800605280000000e900605288001a
:1081d0004c0ae20009003d00401f20006052880068
:1081e0005a0ae20003003a0010002000d052880032
:1081f000020037000000eb00d05288005e0ae20067
:1082000003003200f05280000000e900f0528800c4
:108210004a0ae20003003200505280000000e900e8
:1082200050528800005380000000d00000538800a6
:10823000c3c2bf000080fb004700de000080fb00df
:108240000000e00004003a00005380000000a0009d
:10825000005388000400370000538000e1ff2f0026
:108260000100600000538800105380000000d0001f
:1082700010538800c3c2bf000080fb004600de0030
:108280000080fb00610060000000e00004003a0094
:10829000105380000000a000105388000400370035
:1082a00010538000e1ff2f00010060001053880090
:1082b000640ae2000b003a0000538000e10f400026
:1082c00010003a001000200020538800401f2000ba
:1082d00060538800805380000000e80080538800cd
:1082e00008003700600ae20006003a000000eb00d8
:1082f000205388000000eb00605388000000eb0072
:1083000040538800660ae2000b003a0010538000d8
:10831000e10f400010003a001000200030538800a8
:10832000401f200070538800805380000000e90047
:108330008053880008003700620ae20006003a0015
:108340000000eb00305388000000eb007053880001
:108350000000eb00505388006c0ae2000700320076
:10836000605380000000e900605388006c0ae2005e
:1083700002003a0000052000405388006e0ae20027
:1083800007003200705380000000e900705388003d
:108390006e0ae20002003a000005200050538800f7
:1083a000680ae2000a003200405380000000e90041
:1083b00040538800680ae20005003a0000052000ea
:1083c00040538800805380000000e80080538800fc
:1083d0006a0ae2000a003200505380000000e900ff
:1083e000505388006a0ae20005003a0000052000a8
:1083f00050538800805380000000e90080538800bb
:10840000b05280000000e800b05288000080fa00fe
:108410004f03be004f02be004f01be004f00be0022
:108420003600f900004006000200fa00000f780054
:108430000000eb00c00888001e007800010020004a
:10844000820020000202b8000001eb000283b900a4
:108450000501780006014100830020000388b9006f
:108460000001410082027800e408880086c0a9006b
:1084700021e1a80086c0bf000080fb004600de00ae
:108480000080fb00610060000000e000f9ff3200a6
:1084900021e1a9000080fa00000006000400fa00b3
:1084a000000f78000000eb00100798001e009000fd
:1084b0009e0f500006003100803e2000daff0700ca
:1084c0001e0090000000e80010079800f7ff37003a
:1084d0000080fa00000006003600f800809fbe0011
:1084e000829fbe00849fbe00869fbe000200fa00ed
:1084f00030032000a01088000000eb00000f78007f
:10850000f0cf27009e0f100003003c000000000089
:108510001e0fe800faff370020f02c00801f7800c3
:10852000a6df07008f87e9004207f800c0f12c00a2
:10853000801f7800a1df0700e48757009a0007003a
:10854000ffff37003600f800809fbe00829fbe000c
:10855000849fbe00869fbe000000fa00a0578800de
:10856000b1578800c2578800d3578800e457880065
:10857000f557880006588800175888002858880042
:10858000395888004a5888005b5888006c58880021
:108590007d5888008e5888009f588800a0f22c00d3
:1085a000801f780085df07008f87e900f40af80054
:1085b00020f42c00801f780080df0700e48757003c
:1085c000f60af800c0f42c00801f78007bdf07005b
:1085d000e4875700f80af80060f52c00801f780047
:1085e00076df0700e4875700fa0af80000f62c004f
:1085f000801f780071df0700e4875700fc0af8004d
:10860000a0f62c00801f78006cdf0700e48757007d
:10861000fe0af80040f72c00801f780067df070093
:10862000e4875700000bf800e0f72c00801f78006b
:1086300062df0700e4875700020bf80080f82c0087
:10864000801f78005ddf0700e4875700040bf80007
:1086500020f92c00801f780058df0700e4875700be
:10866000060bf800c0f92c00801f780053df0700cc
:10867000e4875700080bf80060fa2c00801f780090
:108680004edf0700e48757000a0bf80010fb2c00b0
:10869000801f780049df0700e48757000c0bf800c3
:1086a000c0fb2c00801f780044df0700e4875700e0
:1086b0000e0bf80070fc2c00801f78003fdf0700d5
:1086c000e4875700100bf80020fd2c00801f780075
:1086d0003adf0700e4875700120bf800d0fd2c00aa
:1086e000801f780035df0700e48757002e00070061
:1086f000ffff37003600f800809fbe00829fbe005b
:10870000849fbe00869fbe000000fa009f5888002c
:108710000f90200080fe2c00801f780027df0700cc
:108720008f87e900120bf800d0fd2c00801f780025
:1087300022df0700e48757001b000700ffff370018
:108740003600f800809fbe00829fbe00849fbe005e
:10875000869fbe000000fa00e0ff2c00801f78001a
:1087600016df07008f87e9000f000700ffff3700c3
:108770003600f800809fbe00829fbe00849fbe002e
:10878000869fbe000000fa0090a0a9009120a900d9
:1087900030012d00801f780008df07008f87e90077
:1087a00001000700ffff37000000fa00e2f60700b3
:1087b00000032d0099f80700d4c2bf000080fb0021
:1087c00061006000e10f5000fbff3a00cfa2a9005a
:1087d000f9ff3700809fbe00829fbe000400fa00b0
:1087e00090108000004f780040cbbf000040e800b0
:1087f00020479800ae40900000c8bf00000ce10088
:108800000900320002b42000924078000140780054
:108810000080fb0013802000030040001e48780009
:108820008140e800014978000ec2bf000080fb00d3
:108830000000d1000080fb0061006000e10f5000eb
:1088400001003a000e22a9008520a9000080fa004c
:108850004f01be004f00be00004006000000fa00bd
:1088600020042d0030009000a01088000000eb00d4
:10887000601088000000eb00701088008520a900bf
:108880008d20a8000de2a8000f42a8000080fa0089
:10889000000006000200fa00000f780070002000bf
:1088a0009e0f10000200340070002000000f7800be
:1088b00021042d001e0078000000d00001004000bf
:1088c00010007800a01088000080fa000000060068
:1088d0000200fa00004f78000fc2bf000080fb00ca
:1088e0000000d1000080fb0061006000e10f50003b
:1088f000f9ff32001e00fb00f10f200001006000b4
:10890000801088000080fa00000006000000fa00d5
:1089100001b420009140780000c8bf0000c05000a2
:108920000040e9000080fb000080fa000000060023
:108930000000fa000040eb0000e8b70010c0b300f0
:1089400040ebb7000080fa00000006000200fa00c9
:108950000000000000c8bf000040e800004f7800a1
:108960009e40780040cbbf00000ce100f9ff3200d0
:1089700000c8bf000040e80000e8b70000c8bf0022
:108980000080fb0011802000010040001080fb00ef
:108990000080fa00000006000200fa00ebff07006a
:1089a000004f78001e407800c9ff07001e80fb00c2
:1089b0000080fa00000006000600fa006000b8001f
:1089c000008fbe00e1ff07000074a100404798003f
:1089d0004e409000beff0700ce409000f0c2b300b2
:1089e00080cf500016003400ce40900090c3b300fa
:1089f00080cf500012003c001e00be00a2002000ec
:108a00000203b8000001eb000282b9000701780000
:108a100004014100a30020000388b90000014100c7
:108a2000820378004e4090000000fb0001fd2f0003
:108a300001004000cf80de00001f430001974b0083
:108a40004e409000ed4f5000deff3a001e00be0089
:108a50000080fa00000006000400fa00004f7800d1
:108a600090c3b3009e4f100005003e0000cdb30040
:108a70001e4040000000fb00100798001000370067
:108a800060c4b3009e4f100005003e0090ccb300c0
:108a90001e4040000000fb0010079800080037004f
:108aa00060c6b3009e4f100005003e0090cab300a0
:108ab0001e4040000000fb00100798000000370037
:108ac0001e0090000080fa00000006000400fa007a
:108ad0009eff0700204798002e4090007cff070073
:108ae0002e409000dcff0700104798001e409000c9
:108af000004f780095ff0700204798002e40900017
:108b000073ff07002e409000d3ff07001047980026
:108b10009e80fb00000120000088b90080407800a2
:108b20001e40900000cf40001e80fb000080fa0035
:108b3000000006000600fa00881f7800008fbe00c3
:108b400090c0b300504798000040eb0040479800a9
:108b50004e409000e94f500016003c005e409000ef
:108b60000000fb0011902000010440001e00be0028
:108b7000a20020000300200011e9070002c3b30097
:108b8000024c40001e00be00a20020000300200096
:108b90000ee90700008fbe005e4090000040e90033
:108ba000504798004e4090000040e8004047980031
:108bb000e7ff37000040eb000be9b7004f047800f7
:108bc0000080fa00000006000400fa00008fbe00da
:108bd0001e00be00d7ff070001c9bf003cff070011
:108be00002c9bf003aff070003c9bf0038ff0700f2
:108bf00004c9bf0036ff070005c9bf0034ff0700e6
:108c000006c9bf0032ff070007c9bf0030ff0700d9
:108c100008c9bf002eff070009c9bf002cff0700cd
:108c20000ac9bf002aff07000080fa000000060002
:108c30000000fa00d0c3b30025ff070020c4b30032
:108c400023ff0700404c8000ea0f500003003a0069
:108c500000c3b3001eff07000400370088c9bf002f
:108c60006f4060000043b00019ff0700a0c0b300d0
:108c700017ff0700d0c0b30015ff07000080fa00ff
:108c8000000006000000fa00f0c3b30010ff070068
:108c900020c4b3000eff0700a0c0b3000cff070004
:108ca000d0c0b3000aff07000080fa0000000600f1
:108cb0000200fa000000eb00000f780070002000b6
:108cc0009e0f100006003c0080b220009e00400075
:108cd0000040eb00804878001e0fe800f7ff3700e7
:108ce0000000eb00805988000080fa0000000600b8
:108cf0000400fa00004f78001e04e0000c0032006f
:108d0000a0c0b3009e4f10000900320000c2b300a3
:108d10009e4f100006003200c0c2b3009e4f1000ec
:108d200003003200e0c2b3009e4f100003003a007f
:108d30001000200010079800020037000000eb0030
:108d4000100798001e0090000080fa000000060046
:108d50000800fa00edfe07000080fb00000f78001d
:108d60001e00e00046003200f8fe07002047980091
:108d70002e409000deff07000000e00040003a00b7
:108d8000ae409000d0c3b30080cf5000040032004a
:108d9000ae409000f0c3b30080cf500001003a0015
:108da000c3ff07002e409000ed4f500029003a000d
:108db00028cbbf000000fb0030079800d003200044
:108dc000be009000808f50000a003200f0032000a7
:108dd000be009000808f50001c003a0020c4b300f9
:108de000294be30001003a0091ff0700b0ff0700a4
:108df0002300370020c4b300294be30011003a00e0
:108e00002acbbf000000fb006f0060002007980025
:108e10002e009000e90f50000a003c00504c8000ea
:108e2000e10f500007003a00e04c8000e10f5000d5
:108e300004003a002e009000404c880010002000f2
:108e4000305988009aff07000d00370098ff07008f
:108e50000b0037008059800081b2200001004000e3
:108e6000ae4090000148780080598000e60f500025
:108e700003003c00805980000000e8008059880011
:088e80000080fa00000006006a
:020000040000fa
:0200000401f009
:04000000e5ff000018
:020000040000fa
:0200000401f009
:04000400ff7f00007a
:020000040000fa
:0200000401f009
:04000800ffff0000f6
:020000040000fa
:0200000401f009
:04000c00ffff0000f2
:020000040000fa
:0200000401f009
:04001000ffff0000ee
:020000040000fa
:0200000401f009
:04001400ffff0000ea
:020000040000fa
:10000800b84300006c420000a24200007a4300009e
:10001800a0430000b8430000b8430000b843000004
:10002800b8430000b8430000b8430000b8430000dc
:10003800b8430000b84300004a3f00006240000097
:10004800c03e0000ea430000b8430000b843000087
:10005800b8430000b8430000b8430000b8430000ac
:10006800b8430000b8430000b8430000b84300009c
:10007800b8430000b8430000b8430000b84300008c
:10008800b8430000b8430000b8430000b84300007c
:10009800b8430000b8430000b8430000b84300006c
:1000a800b8430000b8430000b8430000b84300005c
:1000b800b8430000b8430000b8430000b84300004c
:1000c800b8430000b8430000b8430000b84300003c
:1000d800b8430000b8430000b8430000b84300002c
:1000e800b8430000b8430000b8430000b84300001c
:0800f800b8430000b84300000a
:020000040000fa
:10010800b84300006c420000a24200007a4300009d
:10011800a0430000b8430000b8430000b843000003
:10012800b8430000b8430000b8430000b8430000db
:10013800b8430000b84300004a3f00006240000096
:10014800c03e0000ea430000b8430000b843000086
:10015800b8430000b8430000b8430000b8430000ab
:10016800b8430000b8430000b8430000b84300009b
:10017800b8430000b8430000b8430000b84300008b
:10018800b8430000b8430000b8430000b84300007b
:10019800b8430000b8430000b8430000b84300006b
:1001a800b8430000b8430000b8430000b84300005b
:1001b800b8430000b8430000b8430000b84300004b
:1001c800b8430000b8430000b8430000b84300003b
:1001d800b8430000b8430000b8430000b84300002b
:1001e800b8430000b8430000b8430000b84300001b
:0801f800b8430000b843000009
:020000040000fa
:108e8800763100002e30000034000000313600003a
:108e98002e310000322e0000323000003038000041
:108ea80000310000323000003020000020000000b7
:108eb80000320000343000003020000020000000a4
:108ec800003400003830000030200000200000008e
:108ed800003900003630000030200000200000007b
:108ee800003100003932000030300000200000005e
:108ef800003300003834000030300000200000004b
:108f08000035000037360000303000002000000037
:108f18000031000031350000323000003020000000
:108f2800003f000021200000312e000038330000ef
:108f38002e350000202000003720000031300000ce
:108f480020310000342000003138000020320000b9
:108f580031200000323400002032000038200000a8
:108f68003f200000dc0500005a0a000082140000bf
:108f780034210000e02e0000803e00002c4c000050
:108f8800e457000090650000307500000a000000fa
:108f98008700000099010000ab020000ba0300003e
:108fa800cc040000df050000ed060000ff0700000c
:108fb80012090000200a0000320b0000450c0000d6
:108fc8000a0d0000576f0000726400007320000053
:108fd8003d200000256400002c200000537500008f
:108fe8006365000073730000203d00002025000029
:108ff800642c00002043000068650000636b0000db
:10900800737500006d2000003d2000002558000009
:10901800000a00000d5700006f7200006473000022
:10902800203d000020250000642c00002053000093
:10903800756300006365000073730000203d000045
:1090480020250000642c0000204300006865000013
:10905800636b0000737500006d2000003d20000068
:1090680025580000002000002020000020200000db
:10907800002000005357000052200000002000008c
:1090880043550000525200000020000054450000e3
:109098004d500000002000003f3f00003f3f00000f
:1090a80000500000575200000050000057520000c6
:1090b8002d2d00002d570000004900000041000040
:1090c80000490000202d00002d2e00002d41000039
:1090d8000050000077720000204f00004646000054
:1090e8002061000066740000657200002025000001
:1090f800692000002000000020200000202000003f
:109108002020000020200000202000002020000057
:109118002020000020200000000a00000d5500005b
:10912800736500007220000073650000747400000d
:10913800696e00006773000020730000617600000c
:1091480065640000207400006f20000045450000a1
:10915800505200004f4d00002c200000506f0000be
:1091680077650000722000006f660000660a000044
:109178000d0000005253000032330000322000007e
:1091880054650000737400002020000020200000b7
:109198002020000000570000616900007469000089
:1091a8006e6700002064000061740000612e0000fa
:1091b8002e2e00002e0000005258000020640000ef
:1091c80061740000612000002000000020200000e1
:1091d800307800000025000069200000000a000027
:1091e8000d0000004a5500004d4100002d500000c0
:1091f8004131000030300000200000002020000035
:109208004f480000324e00004c540000204f000030
:10921800483700005356000020200000005000008e
:109228006f77000065720000204f00004e000000bc
:109238005365000072760000696300006520000035
:109248004d6f000064650000202000002020000011
:1092580000500000757300006820000044490000b9
:10926800535000004c410000592000006e78000067
:10927800740000005075000073680000204f000063
:1092880050450000522000003d20000053610000be
:1092980076650000000a00000d45000045500000fa
:1092a800524f00004d200000636800006563000015
:1092b8006b730000756d0000732c000020430000e4
:1092c800616c0000203d000020250000582c0000a3
:1092d8002044000065660000204300007320000061
:1092e8003d200000255800002c20000046610000a9
:1092f800637400006f72000079200000646500004c
:1093080066610000756c0000742000007265000042
:109318007365000074730000203d000020250000e4
:10932800640000000a0d000045450000505200008e
:109338004f4d00002063000068650000636b00006b
:10934800737500006d20000065720000726f0000e8
:10935800722c000020720000656c00006f61000034
:109368006420000066610000637400006f720000f2
:10937800792000006465000066610000756c0000db
:10938800747300000050000075730000682000002e
:109398005345000054200000666f00007220000052
:1093a80020200000200000006661000063740000b7
:1093b8006f7200007920000064650000666100009b
:1093c800756c000074730000000a00000d0a0000ac
:1093d8000d4a0000554d0000412d0000504100008d
:1093e80031300000302000002f2000000020000055
:1093f8002f200000000a00000d4300006f700000dd
:10940800797200006967000068740000204a000053
:1094180075680000612000004e690000696e000058
:10942800696b00006f7300006b6900002c2000005e
:109438004f480000324e00004c5400000a0d000056
:109448000a0d0000005300007973000074650000e5
:109458006d200000436c00006f6300006b2000006b
:109468003d20000025690000206b0000487a0000bc
:109478000a0d0000000a00000d530000657400008a
:109488002055000041520000542000007573000070
:109498006572000020620000617500006420000011
:1094a8007261000074650000207400006f200000e5
:1094b80023250000692c00002020000025730000ef
:1094c800626400000a0d00000053000057520000bb
:1094d800002000004e2f0000412000000020000066
:1094e800005600000047000031000000473200002d
:1094f800004700003300000047340000002000004f
:109508005354000042590000002000005458000045
:1095180020200000002000004e4f000050200000d6
:10952800002000004f5000004552000000200000bd
:1095380041200000002000004d200000004d0000e8
:10954800487a000000410000757400006f20000098
:10955800426100006e640000204400006574000051
:109568006563000074000000536500006c6500002e
:1095780063740000203d000020000000462d00001c
:10958800736500006e73000065000000545200000f
:10959800583200002020000020000000465400003f
:1095a8002d3800003137000020000000536500000e
:1095b80072690000616c000020500000726f0000aa
:1095c800746f0000636f00006c2000000052000000
:1095d8005332000033320000203d0000200000001c
:1095e8004a5500004d410000545200005832000016
:1095f8000054000065730000742000002020000063
:10960800200000005365000072690000616c0000d2
:1096180020530000706500006564000020200000f1
:109628002020000000420000617500006420000056
:1096380052610000746500003d25000073000000c1
:1096480044690000737000006c2000004272000042
:1096580069670000746800006e650000737300009d
:10966800004c000043440000204200004c20000051
:109678003d20000025690000202000002020000077
:10968800202000000044000069730000706c000096
:1096980061790000204300006f6e000074720000c2
:1096a8006173000074000000436f00006e740000d6
:1096b8007261000073740000203d00002025000046
:1096c80069200000200000005357000052200000cd
:1096d800507200006f740000656300007469000038
:1096e8006f6e000020200000004c0000696d000033
:1096f80069740000203d00002000000020200000c8
:109708002020000000540000656d0000702000005b
:10971800507200006f7400006563000074690000f7
:109728006f6e0000200000004c6900006d690000a9
:10973800742000003d20000025690000200400007e
:10974800432000002020000000460000616e000059
:10975800204300006f6e0000747200006f6c000000
:10976800202000002020000020000000537400008a
:1097780061720000742000003d200000256900008f
:10978800200400004320000020200000000000000a
:10979800200000000001000001020000200300007a
:1097a800030400000402000006060000060600008c
:1097b8000507000007070000447500006d700000f1
:1097c8002045000045500000524f00004d20000089
:1097d800636f00006e740000656e00007473000013
:1097e8000a0d0000000a00000d250000352e0000bb
:1097f8003458000000200000253400005800000004
:109808000a0d00004c610000737400002073000012
:109818007563000063650000737300002063000037
:109828006f640000652000003d20000025580000fe
:10983800200000000a0d00004a5500004d410000bc
:109848002d5400005258000032200000636f0000c1
:1098580070790000726900006768000074200000d9
:109868004f48000037530000562000002620000013
:109878004f480000324e00004c5400000a0d000012
:10988800000a00000d5300006f66000074770000a6
:1098980061720000652000007665000072730000a8
:1098a800696f00006e200000002c0000206300009b
:1098b8006f7000007972000069670000687400002a
:1098c800204a000075680000612000004e69000011
:1098d800696e0000696b00006f7300006b6900001f
:1098e800204f0000483200004e4c0000540a00008f
:1098f8000d0000000a0d0000414400004320000054
:1099080025690000203d00002025000069000000b6
:1099180045450000505200004f4d000020720000e5
:109928006573000065740000206300006f75000017
:109938006e74000065720000206300006c65000012
:1099480061720000656400000a0d0000004c000010
:10995800434400002077000072690000746500002d
:10996800206100007363000069690000200a00009c
:109978000d0000006368000061720000203d0000d7
:1099880020250000780a00000d0000004c4300006c
:109998004420000077720000697400006520000010
:1099a80068650000780a00000d000000203d0000f6
:1099b80020250000630a00000d000000626100001d
:1099c80072200000677200006170000068200000cb
:1099d80074650000737400000a0d0000000a00009e
:1099e8000d5300006f7500006e64000020740000c5
:1099f80065730000742c00002046000043590000e5
:109a08004d4800007a2000002f200000746f0000ed
:109a18006e650000284800007a290000202a00000e
:109a2800203200002c2000006769000076650000e5
:109a380020700000697400006368000020000000c6
:109a48000a0d0000536f0000756e000064200000ce
:109a580074650000737400002c2000006769000022
:109a680076650000206400007572000061740000d3
:109a7800696f00006e2800006d7300002920000047
:109a8800000a00000d530000504900002054000057
:109a980078200000636f00006e740000000a000068
:109aa8000d4600002d730000656e00007365000010
:109ab8002074000065730000742000004f4e000001
:109ac800000a00000d4600002d730000656e0000be
:109ad80073650000207400006573000074200000a6
:109ae8004f660000660000000a0d0000446900008f
:109af8007620000062790000205a0000657200009c
:109b08006f0000004b6500007920000069730000b9
:109b18003a200000256400000a0d000000540000ef
:109b2800727900003a200000566100006c6900005c
:109b380064200000636f00006d6d0000616e00001e
:109b4800647300000a0d0000000000000a0d000008
:109b5800536500007276000069630000652000000c
:109b680026200000636100006c690000627200003a
:109b780061740000696f00006e2000006d6f0000c6
:109b880064650000000a00000d440000495300000d
:109b9800502000003d20000070610000726100004c
:109ba8006d65000074650000722000007365000098
:109bb8006c650000637400002c2000004f5000000a
:109bc80045520000203d000020730000617600002f
:109bd80065200000262000006578000069740000f8
:109be8000053000075700000706c000079200000c0
:109bf8002000000056200000200000004361000003
:109c08006c2000006d7500006c740000203d0000a1
:109c1800202500006c6900002020000020200000a2
:109c28000042000065650000702000006c650000bf
:109c38006e2c0000203000003d4f0000464600001a
:109c4800200000004265000065700000203d000013
:109c580020250000692000006d730000202000000e
:109c680020200000004600006f72000077610000ad
:109c780072640000200000005246000020410000ed
:109c88006d7000002e2000002000000043610000dd
:109c98006c2000006d7500006c740000203d000011
:109ca800202500006c6900002020000000540000fe
:109cb8005258000032200000506f00006c6c000009
:109cc80020520000617400006520000020000000a0
:109cd8005261000074650000203d0000202500004e
:109ce800692000006d730000202000002020000083
:109cf800200000005075000073680000204f00002d
:109d080050450000522000006c6f00006e67000094
:109d1800203d00000066000061630000746f0000d1
:109d2800727900002064000065660000617500001b
:109d38006c7400007300000046610000637400004a
:109d48006f720000792000007365000074750000d0
:109d5800702000006f6b0000000a00000d46000034
:109d680061630000746f00007279000020640000d5
:109d780065660000617500006c74000073200000c7
:109d880072650000737400006f7200006564000063
:109d980000430000616c000069620000722e000040
:109da800205300006176000065640000000a00008e
:109db8000d430000616c00006962000072610000e0
:109dc800746900006f6e0000207300006574000065
:109dd800746900006e670000732000007361000062
:109de8007665000064200000746f000020450000c4
:109df80045500000524f00004d0000000a0d0000c1
:109e080054520000415000003a2000004f730000f7
:109e1800636900006c610000746f0000722000002c
:109e280045720000726f0000720a00000d00000009
:109e38004f530000434300004f4e00002030000005
:109e480078250000580a00000d0000000a0d0000e7
:109e580054520000415000003a20000041640000c4
:109e680064720000657300007320000045720000f2
:109e7800726f0000720a00000d00000057300000e9
:109e88002030000078250000580a00000d0000006e
:109e9800573100002030000078250000580a0000e3
:109ea8000d00000057320000203000007825000027
:109eb800580a00000d000000573300002030000051
:109ec80078250000580a00000d00000057340000f3
:109ed8002030000078250000580a00000d0000001e
:109ee800573500002030000078250000580a00008f
:109ef8000d000000573600002030000078250000d3
:109f0800580a00000d0000005737000020300000fc
:109f180078250000580a00000d000000573800009e
:109f28002030000078250000580a00000d000000cd
:109f3800573900002030000078250000580a00003a
:109f48000d0000005731000030200000307800007c
:109f5800255800000a0d00000057000031310000ac
:109f68002030000078250000580a00000d0000008d
:109f780057310000322000003078000025580000da
:109f88000a0d0000005700003133000020300000a7
:109f980078250000580a00000d0000005731000025
:109fa8003420000030780000255800000a0d000019
:109fb80000570000313500002030000078250000ef
:109fc800580a00000d0000000a0d0000545200005d
:109fd800415000003a200000537400006163000003
:109fe8006b20000045720000726f0000720a0000ca
:109ff8000d0000000a0d00005452000041500000fe
:10a008003a2000004d6100007468000020450000ff
:10a01800727200006f7200000a0d0000000a000052
:10a028000d53000070750000726900006f75000024
:10a0380073200000496e0000746500007272000011
:10a04800757000007420000045720000726f0000f7
:10a05800720a00000d0000002020000020200000ef
:10a0680045720000726f000072200000212000007d
:10a078002020000020200000000000007f010000d8
:10a08800bf0000005f0000002f0000001700000064
:0ca098000b0000000700000003000000a7
:020000040000fa
:10a0a4003e0b00000200000002000000000000005f
:10a0b4000c090000ae00000000000000320b00009c
:10a0c4000600000000000000420a000048000000f2
:10a0d40000000000f40a000020000000000000005e
:10a0e400000800000c01000000000000400b00000c
:10a0f400020000000200000001000000260b000026
:10a104000c00000000000000ba09000088000000f4
:10a11400020000000100000000e00900e109e00085
:10a1240009e00900e009e00009d00900000000008e
:10a13400000000000000000000000000000000001b
:10a1440000000000000000000002080001010800f7
:10a154000a090a00080a08000a080a00080af8009e
:10a1640009000000000000000000000000000000e2
:10a1740000000000000000000000000000000200d9
:10a1840008020200300a31000a300a00300a3000a6
:10a194000a300a00200a000000000000000000004d
:10a1a40000000000000000000000000000000000ab
:10a1b40000000000ba09e200090a0a0000000000d9
:10a1c400000000000000000000000000140b00006c
:10a1d4001200000002000000202b2d00233000009c
:10a1e400010002000004000008001000000000004c
:10a1f4007e0b00000800000002000000686a6c008a
:10a20400747a4c0000000000380b000006000000c7
:10a21400020000000000000000000200420b0000e9
:10a224000200000000000000d20a0000220000002a
:10a234000200000030313200333435003637380044
:10a2440039616200636465006600300031323300b6
:10a25400343536003738390041424300444546001e
:10a26400000000008a0a000048000000020000000c
:10a274000000000000000000244000000000000076
:10a2840000005900400000000000000088c34000a6
:10a29400000000000084d7009741000080e03700f0
:10a2a40079c3410043176e0005b5b500b893460065
:10a2b400f5f93f00e9034f00384d32001d30f90035
:10a2c400487782005a3cbf00737fdd004f1575004c
:10a2d4004c0b000032000000020000004e414e0012
:10a2e400006e61006e0049004e460000696e660013
:10a2f40000303100323334003536370038396100ec
:10a304006263640065660000303132003334350026
:10a3140036373800394142004344450046000000c6
:10a32400440b0000020000000200000000000000d6
:10a33400860b000002000000020000003000000054
:10a34400460b0000020000000200000000000000b4
:10a35400480b0000020000000200000001000000a1
:10a364004a0b000002000000000000000000000092
:00000001FF
